:100000000C9489060C94A6060C94A6060C94A606DD
:100010000C94A6060C94A6060C94A6060C94A606B0
:100020000C94A6060C94A6060C94A6060C94A606A0
:100030000C94A6060C94A6060C94A6060C94A60690
:100040000C94A6060C94A6060C94A6060C94A60680
:100050000C94A6060C94A6060C94A6060C94A60670
:100060000C94A6060C94A6060C94A6060C94A60660
:100070000A696E76616C696420636F6D6D616E6490
:10008000000A562020202056696577207468652074
:10009000636F6465206F6E2074686520637572728B
:1000A000656E746C7920696E736572746564203254
:1000B0003035312F343035312E000A4820202020B1
:1000C0005072696E7420746869732068656C702062
:1000D000646F63756D656E742E000A4120202020C8
:1000E0004175746F20446F776E6C6F616420616E30
:1000F000642050726F6772616D20323035312F3459
:100100003035312E000A4420202020446F776E6C59
:100110006F616420616E20496E74656C204865785B
:100120002066696C6520746F204255524E49542EEA
:10013000000A4320202020436C65617220616E20FC
:1001400041544D454C20323035312F343035312E2D
:10015000000A502020202050726F6772616D20616C
:100160006E2041544D454C20323035312F343035DE
:10017000312E000A4255524E49542048656C700099
:100180000A696E76616C696420636F6D6D616E647F
:10019000000A48202020205072696E74207468691B
:1001A000732068656C7020646F63756D656E742E66
:1001B000000A562020202056696577204675736511
:1001C0006D6170206F6620696E736572746564205E
:1001D00047414C2E000A41202020204175746F2099
:1001E000446F776E6C6F616420616E642050726F33
:1001F0006772616D20612047414C2E000A44202027
:100200002020446F776E6C6F61642061204A454402
:1002100045432066696C6520746F204255524E49F3
:10022000542E000A4320202020436C656172206117
:100230002047414C2E000A502020202050726F672A
:1002400072616D20612047414C2E000A4255524E8A
:1002500049542048656C70000A5665726966696386
:100260006174696F6E204F4B2E000A566572696685
:1002700069636174696F6E204572726F72000A471C
:10028000414C2050726F6772616D6D65642E2E2E29
:10029000566572696679696E672E2E2E000A507255
:1002A0006F6772616D6D696E672047414C2E2E2E0F
:1002B000000A47414C20457261736564000A45722B
:1002C0006173696E672047414C2E2E2E000A4552FD
:1002D000524F5220696E20646F776E6C6F61646953
:1002E0006E67204A454445432E2E2E4175746F702B
:1002F000726F6772616D6D696E672077696C6C20D3
:100300006E6F7420636F6E74696E7565000A4A457E
:1003100044454320446F776E6C6F616420436F6D7A
:10032000706C657465000A4552524F5220696E2008
:10033000646F776E6C6F6164696E67204A454445EF
:1003400043000A4A4544454320446F776E6C6F6111
:100350006420436F6D706C657465000A47414C20E2
:10036000457261736564000A45726173696E672046
:1003700047414C2E2E2E000A696E76616C6964200E
:10038000636F6D6D616E64000A5520202020556EEC
:100390006C6F636B2050494320696620636F64650E
:1003A0002070726F74656374696F6E20656E616230
:1003B0006C65642E000A562020202056696577203F
:1003C00074686520636F6465206F6E2074686520B3
:1003D00063757272656E746C7920696E7365727480
:1003E0006564205049432E000A4820202020507286
:1003F000696E7420746869732068656C7020646F1E
:1004000063756D656E742E000A41202020204175B1
:10041000746F20446F776E6C6F616420616E64202E
:1004200050726F6772616D205049432E000A44205C
:10043000202020446F776E6C6F616420616E2049CC
:100440006E74656C204865782066696C6520746FF1
:10045000204255524E49542E000A4320202020436A
:100460006C6561722061205049432E000A502020A3
:10047000202050726F6772616D2061205049432EB9
:10048000000A4255524E49542048656C70000A4299
:1004900055524E49543E000A47414C323256313093
:1004A000206D6F646520656E61626C6564000A4151
:1004B000746D656C2032303531206D6F6465206558
:1004C0006E61626C6564000A506C656173652063DF
:1004D0006F727265637420616E64207265736574F7
:1004E000204275726E49740A000A4D617962652076
:1004F00074686520636869702069736E2774206969
:100500006E736572746564206F7220746865207301
:10051000776974636820697320696E207468652048
:1005200077726F6E6720706F736974696F6E2E00DB
:100530000A504943206D6F646520656E61626C6589
:1005400064000A57656C636F6D6520746F204255B7
:10055000524E49542076312E31210A507265737300
:100560002027482720666F722068656C702E002E49
:10057000000A4552524F523A20436865636B7375C7
:100580006D20696E76616C696420696E206865789B
:100590002066696C652E000A436865636B20796F7D
:1005A000757220636F6D70696C6572207365747409
:1005B000696E6773206F7220676574206120313621
:1005C000463632382E000A4552524F523A2054686D
:1005D0006973206865782066696C6520686173209E
:1005E0006D6F72652064617461207468616E20743F
:1005F0006865205049433136463632372063616E94
:1006000020686F6C642E00746F2044617461206FE9
:100610007220436F6E666967206D656D6F72792E0B
:1006200020204974206D6967687420616C736F20A5
:10063000626520746F6F2062696720666F72207434
:1006400068697320636869702E000A4552524F52E0
:100650003A2054686973206865782066696C652063
:10066000686173206461746120696E2068696768DD
:10067000206D656D6F7279207468617420646F6598
:1006800073206E6F7420636F72726573706F6E6427
:100690000A000A5761726E696E673A2069676E6F69
:1006A00072696E6720484558207265636F726420D6
:1006B000000A3E000A53696D706C7920636C6561B5
:1006C00072206F7220726570726F6772616D207434
:1006D00068652047414C20746F20636C656172200F
:1006E00074686520736563757269747920667573C3
:1006F00065000A77696C6C206769766520612076F1
:100700006572696669636174696F6E206572726F84
:10071000722061667465722070726F6772616D6DB0
:10072000696E672E000A426563617573652074689F
:1007300069732077696C6C2070726576656E7420C1
:1007400072656164696E67206F75742074686520D6
:1007500066757365206D61702C207468697320471D
:10076000414C000A596F7520686176652063686F97
:1007700073656E20746F2070726F6772616D207484
:100780006865205365637572697479204675736571
:1007900020696E2074686973204A454445432E00E1
:1007A0000A436865636B73756D2057726F6E6700DF
:1007B0000A4E6F204675736520436865636B7375D9
:1007C0006D2070726573656E7420696E204A4544B1
:1007D00045432066696C652E2020436865636B2065
:1007E000636F6D70696C65722073657474696E6790
:1007F00073000A54686973204A4544454320686180
:1008000073207468652077726F6E67206E756D62F5
:100810006572206F662070696E73206F72206E6F34
:100820002070696E206465636C61726174696F6EBB
:100830002E2020497320697420666F722061204742
:10084000414C32325631303F000A54686973204AB5
:100850004544454320686173207468652077726F52
:100860006E67206E756D626572206F6620667573A7
:100870006573206F72206E6F2066757365206465E6
:10088000636C61726174696F6E2E202049732069F8
:100890007420666F7220612047414C3232563130ED
:1008A0003F002E000A3E000A000A50726570617215
:1008B000696E6720746F2070726F6772616D20417E
:1008C000746D656C20323035312F343035312E2E39
:1008D0002E00204F4B2E0056657269666963617465
:1008E000696F6E204661696C656421002E000A56AE
:1008F0006572696679696E672070726F6772616D83
:1009000020646174612E2E2E000A000A556E6B6EF3
:100910006F776E20506172742E2E2E436865636B64
:1009200020436F6E6E656374696F6E73002E204195
:10093000746D656C20343035312E20002E204174CA
:100940006D656C20323035312E200020307800303B
:1009500078000A44657465726D696E696E6720631C
:1009600068697020747970652E2E2E004F4B2E0012
:100970000A436C656172696E6720636869702E2E28
:100980002E2000204F4B2E20002E000A5772697433
:10099000696E6720636869702E2E2E000A5065729A
:1009A000666F726D696E6720746F74616C2062751A
:1009B0006C6B20657261736520746F20636C656178
:1009C0007220636F64652070726F74656374696F01
:1009D0006E2E2E2E000A20434F4E46494720574F79
:1009E0005244203A20000A205553455220494420C1
:1009F0003A20000A000A2044415441203A000A00EB
:100A00000A556E6B6E6F776E205049432C20436FF2
:100A10006E66696720776F7264207761733A000AA7
:100A20005049433136463632382064657465637404
:100A30006564000A504943313646363237206465D2
:100A4000746563746564000A504943313646363232
:100A50003841206465746563746564000A504943D5
:100A60003136463632374120646574656374656497
:100A7000000A49742063616E20616C736F206F6E91
:100A80006C792070726F6772616D20746865206682
:100A90006972737420313238206279746573206F03
:100AA00066204461746120616E64206E6F74206101
:100AB0006C6C203235362062797465732E000A34EE
:100AC0004B206F66206D656D6F7279206F6E20749C
:100AD000686973206465766963652E000A4E6F74D9
:100AE000653A20546869732070726F6772616D6D2A
:100AF00065722063616E206F6E6C792070726F6713
:100B000072616D2074686520666972737420324B5F
:100B1000206F66206D656D6F727920616E64206E46
:100B20006F74207468652077686F6C65000A50499F
:100B300043313646363438412064657465637465E4
:100B4000640049662074686174207761732074685A
:100B500065206F6E6C792070726F626C656D2C20F1
:100B6000646F206E6F7420776F7272792E000A4E58
:100B70004F54453A20546869732070726F677261F0
:100B80006D6D65722063616E6E6F74206469736150
:100B9000626C65204C6F7720566F6C7461676520BE
:100BA00050726F6772616D6D696E670A000A20523C
:100BB0006561643A20000A2053656E743A20000A89
:100BC000566572696669636174696F6E20657272D9
:100BD0006F7220647572696E6720436F6E66696715
:100BE00075726174696F6E2070726F6772616D6D7E
:100BF000696E672E000A50726F6772616D6D696E63
:100C0000672050494320436F6E666967757261744F
:100C1000696F6E20576F72642E2E2E000A56657211
:100C2000696669636174696F6E206572726F7220A4
:100C3000647572696E6720446174612070726F67B9
:100C400072616D6D696E672E000A50726F67726116
:100C50006D6D696E67205049432044617461206D59
:100C6000656D6F72792E2E2E000A436F64652070B9
:100C7000726F74656374696F6E206D61792062654F
:100C800020656E61626C65642E000A566572696645
:100C900069636174696F6E206572726F722064752A
:100CA00072696E672070726F6772616D6D696E67D1
:100CB0002E002E000A50726F6772616D6D696E674B
:100CC000205049432050726F6772616D206D656DD1
:100CD0006F72792E2E2E000A45726173696E67203D
:100CE0005049432064617461206D656D6F72792E87
:100CF0002E2E000A45726173696E672050494320A9
:100D000070726F6772616D206D656D6F72792E2ED6
:100D10002E0011241FBECFEFD0E1DEBFCDBF13E008
:100D2000A0E0B1E0E4EDF8E702C005900D92A23238
:100D3000B107D9F71EE0A2E2B3E001C01D92A73AC5
:100D4000B107E1F70E9407080C94683C0C9400007E
:100D500085B78F7E85BF11B882E084B917B880E46B
:100D60008AB98DEF85B98FEF82B988B98FEB8BB9CE
:100D70000895329B0BC01E9B05C086B120E030E079
:100D8000C901089521E030E0C901089522E030E072
:100D9000C90108952F923F924F925F926F927F9276
:100DA0008F929F92AF92BF92CF92DF92EF92FF927B
:100DB0000F931F93DF93CF93CDB7DEB764970FB632
:100DC000F894DEBF0FBECDBF81EB96E00E942219E2
:100DD0000E9402198A33E1F70E9402190E943B190E
:100DE000582E529460EF56220E9402190E943B191D
:100DF000582A0E9402190E943B19F82EF29450EFD3
:100E0000F5220E9402190E943B19F82A0E94021939
:100E10000E943B19182F1295107F0E9402190E9400
:100E20003B19182B0E9402190E943B19482E42942C
:100E300040EF44220E9402190E943B19482A0F2DBC
:100E4000050D010F040D81E0841588F594E0491625
:100E500009F4BECFA2E04A1609F4BACF82E996E0BF
:100E60000E94221900D000D000D0EDB7FEB7319615
:100E700081E090E08C0F9D1FADB7BEB712969C939A
:100E80008E931197A0E0B1E0B383A28344821582D0
:100E90000E945539EDB7FEB736960FB6F894FEBFEF
:100EA0000FBEEDBFCE0101960E94091991CF5520CA
:100EB00009F469C0812F90E03F2C22243101680E93
:100EC000791E730137E9C32E3EE0D32EC80ED91E1A
:100ED00027E1822E2EE0922E880E991E87E1A82E01
:100EE00086E0B82EA60CB71C13C0D6011C93010FC8
:100EF0000894E11CF11C0894C11CD11C0894811CAD
:100F0000911C0894A11CB11C8E2D86198515D8F54D
:100F10000E9402190E943B19182F1295107F0E94FF
:100F200002190E943B19182BC7018050904440972A
:100F3000E0F2C701805092448138910518F4F40121
:100F40001083D5CFF0E0EF16F8E0FF06D4F58091DE
:100F50002203813019F0D5011C93C9CF80910A0674
:100F60008D3311F08238B9F781E0E81684E0F80695
:100F700090F386EC95E00E94221987E995E00E94A3
:100F800022198FEF27C00E9402190E943B19182FC7
:100F90001295107F0E9402190E943B19182B01958F
:100FA000011751F4B1E04B1611F4552061F18FE6B1
:100FB00095E00E9422190CCF81E795E00E9422194A
:100FC000F1CF8AE496E00E94221987E096E00E9421
:100FD00022198FEF64960FB6F894DEBF0FBECDBF17
:100FE000CF91DF911F910F91FF90EF90DF90CF9005
:100FF000BF90AF909F908F907F906F905F904F9039
:101000003F902F9008950E94021980E0E3CF0F9344
:101010001F9385B78F7E85BF11B812E014B917B83A
:1010200080E48AB98DEF85B90FEF02B908B98FEB6B
:101030008BB91092C50083E38093C40088E180934C
:10104000C10086E08093C2008091C200877F8093B8
:10105000C2000E94021982E495E00E942219329B8C
:101060009AC11E9B7EC186B1109222038EEA94E043
:101070000E94221901B904B917B815B812B80E9414
:10108000891980912203882309F463C1813009F40E
:1010900089C18EE894E00E9422190E9402199927C2
:1010A00087FD90950E945D3C182F0E94FA18809150
:1010B0002203813099F0823009F1133409F4A7C07A
:1010C00014347CF51D3029F3113409F49BC01A3017
:1010D00001F380E790E00E942219DBCF143449F13C
:1010E000153454F51D30A9F21E300CF0B0C01A3082
:1010F00081F287E793E00E942219CBCF143409F4E0
:1011000010C115340CF041C01D3019F21E300CF026
:10111000DEC01A3009F4BDCF80E891E00E942219A8
:10112000B8CF183409F476C019340CF063C0143405
:1011300081F60E94CA06ADCF103509F44EC01135B4
:101140000CF08DC01834A9F681E894E00E942219B1
:101150008CE694E00E94221989E594E00E9422190D
:101160008DE294E00E94221988E094E00E94221906
:1011700088EE93E00E94221985EB93E00E942219E9
:1011800088E893E00E94221984CF103509F478C0D2
:1011900011350CF0B0C0183409F0BECF8BE492E0EA
:1011A0000E94221986E392E00E94221983E292E0D3
:1011B0000E9422198CEF91E00E94221985ED91E0A6
:1011C0000E94221981EB91E00E94221981E991E0AD
:1011D0000E9422195ECF0E94CA060E9471310E94AD
:1011E000A11E97FD56CF0E94882097FD52CF0E94E6
:1011F000E92A4FCF103541F0163509F06ACF0E9429
:10120000791A47CF0E94CA060E944C1B42CF0E9407
:10121000F1193FCF83E791E00E94221981E591E027
:101220000E94221981E391E00E94221985E091E059
:101230000E9422198AED90E00E9422198AEB90E028
:101240000E94221981E890E00E94221922CF1134D5
:1012500011F2133409F04DCF0E9471311ACF1535B8
:1012600099F1163509F045CF0E943D2212CF0E9418
:10127000BC0A892B09F468C08DE093E00E94221912
:1012800080E090E00E94A70D8DEB92E00E94221971
:101290000E94761481EB92E00E9422198DE992E07F
:1012A0000E94221980E090E00E9432158EE792E0C1
:1012B0000E94221981E00E943A10892BD9F18AE616
:1012C00092E00E942219E5CE0E94412DE2CE113417
:1012D00071F2133409F020CF80E090E00E94A70D56
:1012E00087E693E00E9422190E9476148BE593E032
:1012F0000E942219CECE143569F0163509F00CCFB4
:1013000080E090E00E94A70D80E00E943A100E94C9
:101310004A0DBFCE0E944E0F81E090E00E94A70DC3
:10132000B8CE0E94BC0A892B51F082E493E00E945F
:101330002219AFCE88E592E00E942219AACE86E259
:1013400093E00E942219A5CE8DEC92E00E94221912
:10135000A0CEE7E1F6E011922EE0E731F207D9F7EF
:1013600098CE81E08093220380E395E00E942219C9
:1013700084E884B911B90E94262880910A0688233E
:1013800009F07FCE89EE94E00E94221987EC94E068
:101390000E942219FFCF1093220387E994E00E9454
:1013A00022196FCEE7E1F6E08FEF9FE38083918310
:1013B00032962EE0E731F207C9F7E7E1FEE08FEF62
:1013C00081939EE0E739F907D9F7E7E9FEE08FEF6F
:1013D0009FE38083918332962EE0E73AF207C9F7C4
:1013E00058CE892B69F42B9885E0982F9A95F1F7C0
:1013F0002C9A982F9A95F1F72C988A95F1F70895E1
:101400002B9AF2CF181619065CF5672BA9F440E069
:1014100050E035E02B98232F2A95F1F72C9A232FB3
:101420002A95F1F72C98232F2A95F1F74F5F5F4FFC
:101430004817590779F7089540E050E035E02B9AB6
:10144000232F2A95F1F72C9A232F2A95F1F72C9820
:10145000232F2A95F1F74F5F5F4F4817590779F708
:101460000895AF92BF92CF92DF92EF92FF920F93C7
:101470001F93E0EDF7E03197F1F72A98AA2797FD3F
:10148000A095BA2FBC01CD010E94A7365B016C016B
:1014900020E030E04AEF54E40E941D357B018C01CE
:1014A00020E030E040E85FE30E9477368823A4F133
:1014B000C801B70120E03FEF4FE757E40E9417361D
:1014C0001816ACF4C601B50120E030E040E251E46A
:1014D0000E941D350E944733CB01672B79F028EC21
:1014E00030E0F9013197F1F70197D9F707C0C8014A
:1014F000B7010E944733CB010197F1F72A9A80ED9B
:1015000097E00197F1F71F910F91FF90EF90DF9017
:10151000CF90BF90AF90089561E070E0ECCF1816C7
:101520001906DCF440E050E035E013C02B9A232F7D
:101530002A95F1F72C9A232F2A95F1F72C98232F2F
:101540002A95F1F74F5F5F4F4817590731F07595AE
:10155000679560FDEBCF2B98EACF089580B195E0B9
:10156000292F2A95F1F72C9A292F2A95F1F72C98F3
:101570009A95F1F7817008956F927F928F929F9262
:10158000AF92BF92CF92DF92EF92FF920F931F9391
:10159000CF93DF9384EA98E00E9422190E940219F7
:1015A0008230E1F7EE24FF2400E08824AA24BB2443
:1015B0009924CC24DD24E1E06E2E712C0E940219C6
:1015C000182F882329F1133019F11A3209F49AC01F
:1015D000083009F416C109300CF070C0043009F469
:1015E000F1C005300CF094C0023009F4F5C00330AE
:1015F00029F7C12FD0E0CE01C0978A30910508F0BD
:10160000DEC07C0104E00E940219182F8823D9F65D
:101610000E9402190E943B190E9402190E943B1964
:101620000E9402190E943B190E9402190E943B1954
:1016300094E0C91697E1D90609F06EC128E1921627
:1016400009F0ABC1A114B10409F4E9C1EE24FF24EF
:101650008701A1E0B0E060E070E040E050E0769506
:101660006795FA01F595E795F595E795F595E79571
:10167000E75DFC4F808190E0242F277002C0959594
:1016800087952A95E2F780FF02C060587F4F4F5F31
:101690005F4F37E14430530709F4D0C11196A930A8
:1016A000B105E9F6CB01A0E0B0E0E80EF91E0A1F93
:1016B0001B1FA1E0B0E060E070E0D1CF0C3009F476
:1016C00077C00D30D4F50A3009F4BDC00B300CF4EE
:1016D000A9C0C12FD0E0CE01C0970A9708F032C14F
:1016E000C601880F991F880F991F880F991FCC0C6E
:1016F000DD1CC80ED91E80ED9FEFC80ED91ECC0E82
:10170000DD1E5CCF82EA98E00E94221902E056CFEB
:10171000063009F4BEC007300CF4A3C0812F90E05E
:101720000E94553C892B09F049CF103509F45EC160
:10173000163409F46EC102E041CF0E3041F10E3093
:10174000C4F00F3009F03ACF212F30E0C901C09723
:101750000A9708F009C1A294B294B0EFBB22BA2450
:10176000AB22BA2480ED9FEFA80EB91EA20EB31EC5
:1017700025CF812F90E00E94553C892B09F01ECF88
:10178000812F80538230D8F4882E01E017CFC12FEB
:10179000D0E0CE010E94553C892B09F00FCFCE013D
:1017A000C0978A30910508F010C15C010FE006CFA8
:1017B000812F90E00E94553C892B09F0FFCE20E05C
:1017C00030E0B0C0C12FD0E0CE010E94553C892B43
:1017D00009F48BC006E0F2CE812F90E00E94553CC8
:1017E000892B09F0EBCE173409F411C1183408F035
:1017F000DBC0133409F41EC1163409F41DC101E025
:10180000DDCE812F90E00E94553C892B09F0D6CE89
:10181000812F90E0C0970A9790F640ED942E910E9C
:101820000AE0CCCEC12FD0E0CE010E94553C892BDE
:1018300009F0C4CECE01C0978A30910508F0BFCF21
:101840006C010BE0BBCE812F90E0C0970A9708F0A7
:1018500082C01053392D3002C0011124912E980EF0
:10186000ADCEC12FD0E0CE010E94553C892B09F0AE
:10187000A5CE1053123008F0A2CF9E012053304065
:1018800089E293E0B90141EE52E00E944E3901E055
:1018900095CE812F90E00E94553C892B09F08ECE89
:1018A000812F8053823008F08ACFF701F7FCB5C052
:1018B000F595E795F595E795F595E795C70168E006
:1018C00070E00E94F73B103309F493C0E75DFC4FD2
:1018D000930102C0220F331F8A95E2F78081822B89
:1018E00080830894E11CF11C69CECE01C0970A9751
:1018F00008F065CFC701880F991F880F991F880FBF
:10190000991FEE0CFF1CE80EF91E20ED3FEFE20ED2
:10191000F31EEC0EFD1E52CE89E498E00E942219BF
:1019200020E030E0C901DF91CF911F910F91FF902E
:10193000EF90DF90CF90BF90AF909F908F907F906F
:101940006F900895812F90E00E94553C892B09F4F7
:1019500036CF0CE033CE812F90E00E94553C892B8E
:1019600009F42DCF0CE02ACE812F90E00E945D3C3F
:101970009C01815490400697F8F4C5018295929598
:10198000907F9827807F9827F9ECAF2EFFEFBF2E2E
:10199000A20EB31EA80EB91E11CE82EF97E00E94D0
:1019A000221920E030E0BECF1C3409F43FC01135CD
:1019B00009F025CF07E002CE812F90E00E94553C30
:1019C000892B09F4FCCE02E0F9CDCE010E945D3CEA
:1019D0009C0181549040069708F0F1CE19ECA12E9D
:1019E0001FEFB12EA20EB31E0FE0E8CD08E0992440
:1019F000E5CDE75DFC4F930102C0220F331F8A95AE
:101A0000E2F7C90180952081822380836ACF0DE0AF
:101A1000D5CD09E0CC24DD24D1CD379649CF80EB5C
:101A200097E00E94221920E030E07CCFEE24FF24D2
:101A300003E0C4CD0EE0C2CD05E0C0CD88E090E06B
:101A40008A1B9B0B02C0769567958A95E2F76E0D0F
:101A50007F1DA616B70631F481E0881651F021E00B
:101A600030E060CF80EA97E00E94221920E030E069
:101A700059CF83E697E00E94221985E297E00E9401
:101A8000221982EF96E00E94221984EB96E00E94D0
:101A90002219E5CFCF92DF92EF92FF920F931F931F
:101AA000DF93CF93CDB7DEB728970FB6F894DEBF9C
:101AB0000FBECDBF00E010E080E090E07E01089412
:101AC000E11CF11CFBE0CF2EF1E0DF2E28C000D09E
:101AD00000D000D0EDB7FEB73196ADB7BEB71296C5
:101AE000FC92EE921197D382C282D801A75DBC4FBF
:101AF0008C91848315820E9455398DB79EB70696C6
:101B00000FB6F8949EBF0FBE8DBFC7010E94091982
:101B10000F5F1F4FC801A2E0013E1A0749F08F7105
:101B20009070892BA1F687EA98E00E942219CFCF06
:101B300028960FB6F894DEBF0FBECDBFCF91DF91D0
:101B40001F910F91FF90EF90DF90CF9008950F932A
:101B50001F93DF93CF93CDB7DEB7C456D0400FB6F7
:101B6000F894DEBF0FBECDBFAC0180910C0690E0B3
:101B70008F7090708530910509F4CFC020910E06CA
:101B80008130910509F4D7C0823091050CF4E6C08C
:101B90008230910509F4DDC0039709F4D3C084E6CF
:101BA00090E0909324038093230388EC90E090933B
:101BB000260380932503452B61F4CC59DF4F0FB6E4
:101BC000F894DEBF0FBECDBFCF91DF911F910F9173
:101BD000089540912703509128036DB77EB76A504E
:101BE00070400FB6F8947EBF0FBE6DBFEDB7FEB765
:101BF00031968E010F5F1F4FADB7BEB712961C9383
:101C00000E9311978FE091E093838283CA0157FD71
:101C1000AFC0959587959595879595838483242F57
:101C2000217089E128029001112456954795417051
:101C3000507082E390E0BC01469FC001479F900D29
:101C4000569F900D1124280F822F992787FD90957C
:101C50009783868384E690E0918780870E94553938
:101C60008DB79EB70A960FB6F8949EBF0FBE8DBF74
:101C7000C8010E940919ADB7BEB75C970FB6F894BA
:101C8000BEBF0FBEADBFEDB7FEB7319612961C9327
:101C90000E93119788E391E09383828380910B06E2
:101CA0008483158280910C068683178280910D06AD
:101CB0008087118680910E068287138680910F0699
:101CC0008487158680911006868717868091110675
:101CD000808B118A80911206828B138A8091130661
:101CE000848B158A80911406868B178A809115063D
:101CF000808F118E80911606828F138E0E94553927
:101D00006DB77EB7645E7F4F0FB6F8947EBF0FBE8F
:101D10006DBFC8010E94091950CF809110068695A9
:101D200090E08F7190700A96880F991F9093280306
:101D30008093270334CF8FE390E090932803809320
:101D400027032DCF88E390E0909328038093270307
:101D500026CF2F3879F08AE390E0F6CF892B09F06F
:101D60001ECF82E490E0909328038093270317CF3F
:101D700003964FCF8CE390E0E7CFBC015B9840988F
:101D800041982D982E982D9820E030E045E02B9832
:101D9000842F8A95F1F72C9A842F8A95F1F72C9845
:101DA000842F8A95F1F72F5F3F4F2438310579F75B
:101DB00060FF68C02B9A85E0282F2A95F1F72C9AAE
:101DC000282F2A95F1F72C988A95F1F7AB015595B4
:101DD000479540FF61C02B9A85E0282F2A95F1F79F
:101DE0002C9A282F2A95F1F72C988A95F1F755957A
:101DF000479540FF4FC02B9A85E0282F2A95F1F791
:101E00002C9A282F2A95F1F72C988A95F1F7559559
:101E1000479540FF3DC02B9A85E0282F2A95F1F782
:101E20002C9A282F2A95F1F72C988A95F1F7559539
:101E3000479540FF2BC02B9A85E0282F2A95F1F774
:101E40002C9A282F2A95F1F72C988A95F1F741FFC3
:101E50001BC02B9A85E0982F9A95F1F72C9A982F12
:101E60009A95F1F72C988A95F1F780ED97E0FC01AF
:101E70003197F1F72A98FC013197F1F72A9A0197E7
:101E8000F1F708952B9897CF2B98E4CF2B98D4CFC8
:101E90002B98C2CF2B98B0CF2B989ECF11B882E051
:101EA00084B917B880E48AB99FEF92B98DEF85B9EC
:101EB00098B98BB18F6B8BB985E38A95F1F75E9AF0
:101EC00020E030E048EC50E0CA010197F1F72F5FC5
:101ED0003F4F83E0283E3807B9F720E23EE4C901CE
:101EE0000197F1F712B884E085B918B88BB1807406
:101EF0008BB98EEF81B98FEF84B983E087B98CED10
:101F00008AB980E49CE90197F1F72898C901019703
:101F1000F1F78AE390E00E94BD0EEBE0F6E025E0E9
:101F2000108280B1922F9A95F1F72C9A922F9A9560
:101F3000F1F72C98922F9A95F1F780FF03C08081DA
:101F40008160808380B1922F9A95F1F72C9A922F1D
:101F50009A95F1F72C98922F9A95F1F780FF03C08C
:101F600080818260808380B1922F9A95F1F72C9ABC
:101F7000922F9A95F1F72C98922F9A95F1F780FF6E
:101F800003C080818460808380B1922F9A95F1F79D
:101F90002C9A922F9A95F1F72C98922F9A95F1F707
:101FA00080FF03C080818860808380B1922F9A95E2
:101FB000F1F72C9A922F9A95F1F72C98922F9A95E7
:101FC000F1F780FF03C080818061808380B1922F10
:101FD0009A95F1F72C9A922F9A95F1F72C98922FC7
:101FE0009A95F1F780FF03C080818062808380B181
:101FF000922F9A95F1F72C9A922F9A95F1F72C98A7
:10200000922F9A95F1F780FF03C0808180648083CE
:1020100080B1922F9A95F1F72C9A922F9A95F1F719
:102020002C98922F9A95F1F780FF03C080818068E9
:102030008083319686E0E531F80709F071CF80E9B9
:1020400091E00197F1F711B882E084B917B880E404
:102050008AB99FEF92B98DEF85B998B98BB18F6B23
:102060008BB980E29EE40197F1F75E9885E38A954B
:10207000F1F708952F923F924F925F926F927F9265
:102080008F929F92AF92BF92CF92DF92EF92FF9288
:102090000F931F93DF93CF93CDB7DEB728970FB67B
:1020A000F894DEBF0FBECDBF888711B882E084B937
:1020B00017B880E48AB99FEF92B98DEF85B998B9C6
:1020C0008BB18F6B8BB985E38A95F1F75E9A20E02F
:1020D00030E048EC50E0CA010197F1F72F5F3F4F25
:1020E00083E0283E3807B9F720E23EE4C9010197B2
:1020F000F1F712B884E085B918B88BB180748BB948
:102100008EEF81B98FEF84B983E087B98CED8AB9FE
:1021100080E49CE90197F1F72898C9010197F1F74C
:102120008091A4019091A501181619060CF0DAC34C
:10213000AA24BB2422243324CC2495E0D92E80ED7C
:10214000482E87E0582E01E0602E712C5B98409855
:1021500041982D982E982D9820E030E02B988D2DC9
:102160008A95F1F72C9A8D2D8A95F1F72C988D2D63
:102170008A95F1F72F5F3F4F2438310579F7A0FE9C
:1021800046C12B9A8D2D8A95F1F72C9A8D2D8A9523
:10219000F1F72C988D2D8A95F1F7950135952795B6
:1021A00020FF3DC12B9A8D2D8A95F1F72C9A8D2D0C
:1021B0008A95F1F72C988D2D8A95F1F7359527950D
:1021C00020FF2BC12B9A8D2D8A95F1F72C9A8D2DFE
:1021D0008A95F1F72C988D2D8A95F1F735952795ED
:1021E00020FF19C12B9A8D2D8A95F1F72C9A8D2DF0
:1021F0008A95F1F72C988D2D8A95F1F735952795CD
:1022000020FF07C12B9A8D2D8A95F1F72C9A8D2DE1
:102210008A95F1F72C988D2D8A95F1F721FFF5C05D
:102220002B9A8D2D8A95F1F72C9A8D2D8A95F1F7A1
:102230002C988D2D8A95F1F7C2010197F1F72A9814
:10224000C2010197F1F72A9AC2010197F1F7809034
:10225000A6019090A701181419040CF040C0E0905A
:10226000A401F090A5019885992309F0DAC000E057
:1022700010E0E09EC001E19E900DF09E900D1124B3
:102280008A0D9B1D9C0197FDBDC035952795359501
:1022900027953595279568E070E00E94F73B482F19
:1022A00080B19D2D9A95F1F72C9A9D2D9A95F1F775
:1022B0002C989D2D9A95F1F780FF96C0C30102C01E
:1022C000880F991F4A95E2F7F901E75DFC4F90816D
:1022D000982B90830F5F1F4F0815190554F208942F
:1022E000A11CB11C8091A4019091A501A816B9066A
:1022F0000CF42CCF8091A8019091A9010E94BD0EF1
:102300008091AC019091AD01181619060CF059C1DD
:10231000A885AA2309F414C100E010E0A5E0DA2E94
:10232000F1E0AF2EB12C4E010894811C911CE2E625
:102330006E2EE1E07E2E2BC0C501042E02C0880F58
:10234000991F0A94E2F7C82A8C2D992787FD90954A
:10235000F701E75DFC4F208130E082279327042EB0
:1023600002C0959587950A94E2F780FD91C20F5FB0
:102370001F4F8091AC019091AD01880F991F880F7C
:10238000991F880F991F081719070CF01AC180911F
:10239000AA019091AB01800F911FFC0197FD4BC2E8
:1023A0007F01F594E794F594E794F594E79468E059
:1023B00070E00E94F73BAC0180B19D2D9A95F1F73A
:1023C0002C9A9D2D9A95F1F72C989D2D9A95F1F7C1
:1023D00080FDB2CFC501042E02C0880F991F0A9458
:1023E000E2F78095C822B0CFC30102C0880F991FC1
:1023F0004A95E2F7982F9095F901E75DFC4F8081AF
:10240000982367CF295F3F4F40CF2B980ACF2B9857
:10241000B9CE2B98F8CE2B98E6CE2B98D4CE2B980D
:10242000C2CE00E010E029C0C301042E02C0880F14
:10243000991F0A94E2F7C82A8C2D992787FD909559
:10244000F701E75DFC4F208130E082279327042EBF
:1024500002C0959587950A94E2F780FD40C00F5F12
:102460001F4F8091A6019091A701081719070CF042
:1024700036CFE090A401F090A5010E9DC0010F9D04
:10248000900D1E9D900D11248A0D9B1DFC0197FD42
:1024900024C07F01F594E794F594E794F594E794CC
:1024A00068E070E00E94F73BAC0180B19D2D9A95E9
:1024B000F1F72C9A9D2D9A95F1F72C989D2D9A95D0
:1024C000F1F780FDB1CFC301042E02C0880F991F20
:1024D0000A94E2F78095C822AFCF3796DACF00D0C2
:1024E00000D000D0EDB7FEB7319681E090E08C0FC0
:1024F0009D1FADB7BEB712969C938E931197A2E61F
:10250000B1E0B383A283C701880F991F880F991F79
:10251000880F991F840F951F958384830E945539D6
:102520008DB79EB706960FB6F8949EBF0FBE8DBFAF
:10253000CE0101960E94091931E0232E312C8FCF54
:1025400000E010E05C01AA0CBB1CAA0CBB1CAA0C8E
:10255000BB1C95E0F92E81E0882E912C8091AA0178
:102560009091AB01800F911F9C0197FD61C1359542
:102570002795359527953595279568E070E00E9459
:10258000F73B482F80B19F2D9A95F1F72C9A9F2DFC
:102590009A95F1F72C989F2D9A95F1F780FF38C105
:1025A000C40102C0880F991F4A95E2F7F901E75D5F
:1025B000FC4F9081982B90830F5F1F4F0A151B05CE
:1025C0006CF28091B60180FF13C15B9A81FF0EC14E
:1025D000409A82FF09C1419A83FF04C12F9A84FF68
:1025E000FCC02E9A85FDFCC02D9880ED97E0FC0183
:1025F0003197F1F72A98E0EAFFE03197F1F72A9A4C
:102600000197F1F7A090BA01B090BB011A141B0416
:102610000CF0AFC09885992309F469C000E010E080
:10262000B5E0DB2EA1E0AA2EB12C4E010894811C4E
:10263000911CF2E66F2EF1E07F2E25C0C501042E1D
:1026400002C0880F991F0A94E2F7C82A8C2D992797
:1026500087FD9095F701E75DFC4F208130E08227F0
:102660009327042E02C0959587950A94E2F780FD82
:10267000E6C00F5F1F4F8091BA019091BB01081710
:1026800019070CF076C0C801880F991FE091B801B6
:10269000F091B901E80FF91F408151819A01C901F8
:1026A00037FDCBC07C01F594E794F594E794F5945D
:1026B000E794CA0168E070E00E94F73BAC0180B18A
:1026C0009D2D9A95F1F72C9A9D2D9A95F1F72C98BE
:1026D0009D2D9A95F1F780FDB1CFC501042E02C062
:1026E000880F991F0A94E2F78095C822AFCF00E0C7
:1026F00010E0C090B801D090B90135E0F32E21E090
:10270000822E912CF801EE0FFF1FEC0DFD1D408174
:1027100051819A01C90137FD89C09C0135952795E2
:102720003595279535952795CA0168E070E00E9498
:10273000F73B482F80B19F2D9A95F1F72C9A9F2D4A
:102740009A95F1F72C989F2D9A95F1F780FF52C03A
:10275000C40102C0880F991F4A95E2F7F901E75DAD
:10276000FC4F9081982B90830F5F1F4F0A151B051C
:102770004CF280E991E00197F1F711B882E084B959
:1027800017B880E48AB99FEF92B98DEF85B998B9EF
:102790008BB18F6B8BB980E29EE40197F1F75E9865
:1027A00085E38A95F1F7C10128960FB6F894DEBF4C
:1027B0000FBECDBFCF91DF911F910F91FF90EF9092
:1027C000DF90CF90BF90AF909F908F907F906F9051
:1027D0005F904F903F902F9008952E9885FF04CFE3
:1027E0002D9A03CF2D98FBCE4198F6CE4098F1CE8E
:1027F0005B98ECCEC40102C0880F991F4A95E2F79E
:10280000982F9095F901E75DFC4F80819823ABCF1D
:10281000C40102C0880F991F4A95E2F7982F90953E
:10282000F901E75DFC4F80819823C5CE079675CFEF
:10283000295F3F4F9CCE3796B3CD079633CF00D05C
:1028400000D000D0EDB7FEB73196ADB7BEB7129647
:102850009C928E92119773826282EE0CFF1CEE0C9A
:10286000FF1CEE0CFF1CE40EF51EF582E4820E94B4
:1028700055398DB79EB706960FB6F8949EBF0FBE1A
:102880008DBFC4010E94091941E0242E312CF1CEE4
:1028900000D000D000D0EDB7FEB73196ADB7BEB7CF
:1028A00012969C928E92119773826282C701880F52
:1028B000991F880F991F880F991F840F951F958363
:1028C00084830E9455398DB79EB706960FB6F8944B
:1028D0009EBF0FBE8DBFC4010E94091951E0252E75
:1028E000312C45CD22243324CC2404CDAF92BF9289
:1028F000CF92DF92EF92FF920F931F9311B882E075
:1029000084B917B880E48AB99FEF92B98DEF85B981
:1029100098B98BB18F6B8BB985E38A95F1F75E9A85
:1029200020E030E048EC50E0CA010197F1F72F5F5A
:102930003F4F83E0283E3807B9F720E23EE4C90163
:102940000197F1F712B884E085B918B88BB180749B
:102950008BB98EEF81B98FEF84B983E087B98CEDA5
:102960008AB980E49CE90197F1F7289AC901019797
:10297000F1F75B9A4098419A2F9A2E9A2D9A80ED02
:1029800097E00197F1F72A9860912503709126034B
:10299000882777FD8095982F0E94A7365B016C01F0
:1029A00020E030E04AEF54E40E941D357B018C01A9
:1029B00020E030E040E85FE30E947736882304F1AE
:1029C000C801B70120E03FEF4FE757E40E941736F8
:1029D00018160CF042C0C601B50120E030E040E21C
:1029E00051E40E941D350E944733CB01672B69F0EB
:1029F00028EC30E0F9013197F1F70197D9F705C0DC
:102A000061E070E0CB010197F1F72A9A80ED97E041
:102A10000197F1F780E991E00197F1F711B882E0B1
:102A200084B917B880E48AB99FEF92B98DEF85B960
:102A300098B98BB18F6B8BB980E29EE40197F1F767
:102A40005E9885E38A95F1F71F910F91FF90EF90C3
:102A5000DF90CF90BF90AF900895C801B7010E945A
:102A60004733D0CF2F923F924F925F926F927F92D7
:102A70009F92AF92BF92CF92DF92EF92FF920F930D
:102A80001F93DF93CF93CDB7DEB728970FB6F89497
:102A9000DEBF0FBECDBF9A83898311B882E084B9AF
:102AA00017B880E48AB99FEF92B98DEF85B998B9CC
:102AB0008BB18F6B8BB985E38A95F1F75E9A20E035
:102AC00030E048EC50E0CA010197F1F72F5F3F4F2B
:102AD00083E0283E3807B9F720E23EE4C9010197B8
:102AE000F1F712B884E085B918B88BB180748BB94E
:102AF0008EEF81B98FEF84B983E087B98CED8AB905
:102B000080E49CE90197F1F7289AC9010197F1F750
:102B10005B98409841982D982E982D982090A4016C
:102B20003090A501121413040CF059C36090A60153
:102B30007090A701A0912303B0912403B887AF83BD
:102B400044245524CD01AA2797FDA095BA2F8B8345
:102B50009C83AD83BE8375E0972E16141704ACF5E5
:102B6000A981BA81AB2B09F09BC2720100E010E091
:102B7000A701F701F7FC86C2F595E795F595E7956E
:102B8000F595E795E75DFC4F208130E0CA0168E0EC
:102B900070E00E94F73B02C0359527958A95E2F7D1
:102BA00020FF6EC22B9A892D8A95F1F72C9A892DD8
:102BB0008A95F1F72C98892D8A95F1F70F5F1F4FB1
:102BC000E20CF31C061517059CF240FC5FC22B9823
:102BD000892D8A95F1F72C9A892D8A95F1F72C98F1
:102BE000892D8A95F1F792013595279520FD56C2DA
:102BF0002B98892D8A95F1F72C9A892D8A95F1F7D2
:102C00002C98892D8A95F1F73595279520FD44C29A
:102C10002B98892D8A95F1F72C9A892D8A95F1F7B1
:102C20002C98892D8A95F1F73595279520FD32C28C
:102C30002B98892D8A95F1F72C9A892D8A95F1F791
:102C40002C98892D8A95F1F73595279520FD20C27E
:102C50002B98892D8A95F1F72C9A892D8A95F1F771
:102C60002C98892D8A95F1F721FF0EC22B9A892D78
:102C70008A95F1F72C9A892D8A95F1F72C98892D50
:102C80008A95F1F72B9880ED97E00197F1F72A9854
:102C90006B817C818D819E810E94A7365B016C01D6
:102CA00020E030E04AEF54E40E941D357B018C01A6
:102CB00020E030E040E85FE30E94773688230CF4A0
:102CC0000BC2C801B70120E03FEF4FE757E40E9475
:102CD000173618160CF0F8C1C601B50120E030E037
:102CE00040E251E40E941D350E944733CB01672B1F
:102CF00031F0E8ECF0E03197F1F70197D1F72A9A3B
:102D000080ED97E00197F1F70894411C511C4214A3
:102D100053040CF422CF0091AC011091AD01000FCF
:102D2000111F000F111F000F111F101611060CF0BC
:102D300039C0E090AA01F090AB0129813A81232BA0
:102D400009F0CFC1CC24DD2445E0C6018E0D9F1DC6
:102D5000FC0197FDFEC1F595E795F595E795F5958D
:102D6000E795E75DFC4F208130E068E070E00E946D
:102D7000F73B02C0359527958A95E2F720FFE7C11A
:102D80002B9A842F8A95F1F72C9A842F8A95F1F744
:102D90002C98842F8A95F1F70894C11CD11CC01679
:102DA000D1069CF2061517050CF4B3C12091A801B9
:102DB0003091A90120FD93C12B9885E0982F9A9519
:102DC000F1F72C9A982F9A95F1F72C988A95F1F7AC
:102DD0003595279520FDC9C12B9885E0982F9A95A8
:102DE000F1F72C9A982F9A95F1F72C988A95F1F78C
:102DF0003595279520FDB7C12B9885E0982F9A959A
:102E0000F1F72C9A982F9A95F1F72C988A95F1F76B
:102E10003595279520FDA5C12B9885E0982F9A958B
:102E2000F1F72C9A982F9A95F1F72C988A95F1F74B
:102E30003595279520FD93C12B9885E0982F9A957D
:102E4000F1F72C9A982F9A95F1F72C988A95F1F72B
:102E500021FF83C12B9A85E0982F9A95F1F72C9A40
:102E6000982F9A95F1F72C988A95F1F72B9880ED89
:102E700097E00197F1F72A98AF81B885BD018827BF
:102E800077FD8095982F0E94A7362B013C0120E00A
:102E900030E04AEF54E40E941D355B016C0120E0F4
:102EA00030E040E85FE30E94773688230CF491C15C
:102EB000C601B50120E03FEF4FE757E40E94173607
:102EC00018160CF076C1C301B20120E030E040E2F8
:102ED00051E40E941D350E944733CB01672B39F026
:102EE00028EC30E0F9013197F1F70197D9F72A9AE8
:102EF00080ED97E00197F1F78091B60180FF42C124
:102F00005B9A81FF3DC1409A82FF38C1419A83FF9D
:102F100033C12F9A84FF2BC12E9A85FD2BC12D988A
:102F2000E090BA01F090BB011E141F040CF041C0E8
:102F30002091B8013091B901E981FA81EF2B09F0B4
:102F400023C1190100E010E035E0932ED1014C912E
:102F500011965C91CA01FC0197FDFDC0F595E795BE
:102F6000F595E795F595E795E75DFC4F208130E015
:102F7000CA0168E070E00E94F73B02C035952795D2
:102F80008A95E2F720FFE1C02B9A892D8A95F1F707
:102F90002C9A892D8A95F1F72C98892D8A95F1F72D
:102FA0000F5F1F4FE2E0F0E02E0E3F1E0E151F05D3
:102FB0006CF22B9880ED97E00197F1F72A98C60103
:102FC000B50120E030E040E85FE30E9477368823D7
:102FD0000CF402C1C601B50120E03FEF4FE757E412
:102FE0000E94173618160CF0ECC0C301B20120E0A5
:102FF00030E040E251E40E941D350E944733CB018E
:10300000672B39F028EC30E0F9013197F1F701979F
:10301000D9F72A9A80ED97E00197F1F780E991E0DE
:103020000197F1F711B882E084B917B880E48AB942
:103030009FEF92B98DEF85B998B98BB18F6B8BB932
:1030400080E29EE40197F1F75E9885E38A95F1F7B7
:1030500028960FB6F894DEBF0FBECDBFCF91DF919B
:103060001F910F91FF90EF90DF90CF90BF90AF90A6
:103070009F907F906F905F904F903F902F9008951A
:103080002B9891CD379678CD2B98F1CD2B9AA0CD5A
:103090002B9ADFCD2B9ACDCD2B9ABBCD2B9AA9CDD8
:1030A00020E030E02B9A892D8A95F1F72C9A892D12
:1030B0008A95F1F72C98892D8A95F1F72F5F3F4F6C
:1030C000261537057CF381CDC801B7010E9447332F
:1030D000CB010197F1F713CE61E070E0F9CF2B9AA5
:1030E0006CCE20E030E095E02B9A892F8A95F1F79D
:1030F0002C9A892F8A95F1F72C98892F8A95F1F7C8
:103100002F5F3F4F201731077CF3061517050CF092
:103110004DCEA301401B510B141615060CF046CEE4
:1031200020E030E095E02B98892F8A95F1F72C9AD2
:10313000892F8A95F1F72C98892F8A95F1F72F5FBF
:103140003F4F2417350779F731CE2B981ECF2B9898
:1031500018CE379600CE379601CF2B987CCE2B9A7F
:103160006CCE2B9A5ACE2B9A48CE2B9A36CE2E98CE
:1031700085FFD5CE2D9AD4CE2D98CCCE4198C7CEF2
:103180004098C2CE5B98BDCE20E030E095E02B9A0F
:10319000892F8A95F1F72C9A892F8A95F1F72C9827
:1031A000892F8A95F1F72F5F3F4F2E153F057CF34E
:1031B00000CFC601B5010E944733CB010197F1F75B
:1031C00096CEC601B5010E944733CB010197F1F7B6
:1031D00020CF61E070E0F1CF61E070E0F6CF609069
:1031E000A6017090A701E0912303F0912403F887D2
:1031F000EF8391CD982F8091C00085FFFCCF9093F5
:10320000C60008958091C00087FFFCCF8091C60062
:103210000895FC019081992369F02DE09A3059F0CE
:1032200031968091C00085FFFCCF9093C6009081BD
:103230009923A1F708958091C00085FFFCCF2093CA
:10324000C600EECFFC019491992369F02DE09A30ED
:1032500059F08091C00085FFFCCF9093C600319655
:1032600094919923A1F708958091C00085FFFCCF28
:103270002093C600EECF813414F087530895805315
:1032800008950F931F93DF93CF9300D00F92CDB784
:10329000DEB700D000D000D0EDB7FEB731968E017A
:1032A0000F5F1F4FADB7BEB712961C930E931197C9
:1032B00024E032E033832283848315820E945539CF
:1032C00099812DB73EB72A5F3F4F0FB6F8943EBFA6
:1032D0000FBE2DBF992371F0F8012DE09A3091F0C7
:1032E00031968091C00085FFFCCF9093C6009081FD
:1032F0009923A1F70F900F900F90CF91DF911F911D
:103300000F9108958091C00085FFFCCF2093C600E7
:10331000E7CF2F9A82E0982F9A95F1F72F988A9508
:10332000F1F708950F931F93CF93DF938EEE98E0FC
:103330000E94221911B815B88AE18A95F1F785B172
:10334000816485B985B18F7C85B985B18C6085B97B
:1033500085E08A95F1F7C0E0D0E012E005E017C003
:1033600080B1FE01E95EF94F9081981701F52F9A1F
:10337000812F8A95F1F72F98812F8A95F1F7802F69
:103380008A95F1F7219688E0C030D807E9F0CE01A0
:103390008F779070892B21F78CEE98E00E9422198C
:1033A00080B1FE01E95EF94F9081981701F387ED36
:1033B00098E00E94221915B88FEF81B912B8DF91F9
:1033C000CF911F910F91089515B88FEF81B912B861
:1033D00082ED98E00E942219DF91CF911F910F9109
:1033E000089580E799E00E94221915B885B181649B
:1033F00085B92D9A85B1837E85B98AE18A95F1F7E1
:10340000299A80E28A95F1F72E9880E29EE4FC01E9
:103410003197F1F72E9AFC013197F1F7299801972E
:10342000F1F715B88CE699E00E9422190895FF92F1
:103430000F931F93CF93DF938BE899E00E9422199B
:1034400015B812B88AE18A95F1F785B1816485B91A
:103450002D9885B18C6185B985E08A95F1F7299A17
:1034600080E58A95F1F7C0E0D0E005E08AE1F82E2A
:1034700012E0CE018F779070892B09F435C0FE01E0
:10348000E95EF94F808182B9802F8A95F1F72E98F5
:103490008F2D8A95F1F72E9A3099FECF309BFECF73
:1034A0002F9A812F8A95F1F72F98812F8A95F1F71E
:1034B000802F8A95F1F7219688E0C030D807C9F6A9
:1034C00080E29EE4FC013197F1F729980197F1F72A
:1034D00015B812B883E899E00E942219DF91CF91C4
:1034E0001F910F91FF90089589E899E00E94221999
:1034F000C6CFAF92BF92CF92DF92EF92FF920F931F
:103500001F93DF93CF93CDB7DEB72A970FB6F8940A
:10351000DEBF0FBECDBF11B815B88AE18A95F1F7AD
:1035200085B1816485B985B18F7C85B985B18C60A1
:1035300085B985E08A95F1F700E010E06E01089406
:10354000C11CD11C39E0A32E32E0B32E22E0F22EB2
:1035500095E0E92E14C080B10E9441192F9A8F2D59
:103560008A95F1F72F988F2D8A95F1F78E2D8A95F0
:10357000F1F70F5F1F4F98E00030190739F1C801CC
:103580008F719070892B39F789E099E00E94221998
:1035900000D000D000D0EDB7FEB73196ADB7BEB7C2
:1035A0001296DC92CE921197B382A2821583048385
:1035B0000E9455398DB79EB706960FB6F8949EBFF8
:1035C0000FBE8DBFC6010E940919C5CF15B88FEF78
:1035D00081B912B82A960FB6F894DEBF0FBECDBFE0
:1035E000CF91DF911F910F91FF90EF90DF90CF90DF
:1035F000BF90AF9008950F931F9382E599E00E94CA
:10360000221911B815B88AE18A95F1F785B181645C
:1036100085B985B1837C85B98FE499E00E94221930
:1036200015E0812F8A95F1F700B1802F0E94411992
:103630008BE499E00E9422192F9A82E0982F9A95A4
:10364000F1F72F988A95F1F71A95F1F710B1812FBC
:103650000E94411915B88FEF81B912B80E3151F09F
:103660008BE099E00E94221921E030E0C9011F910E
:103670000F910895113249F0113491F78DE299E0DC
:103680000E94221920E030E0F1CF8CE399E00E9403
:10369000221920E030E0EACFFF920F931F93CF93DF
:1036A000DF9389EA98E00E9422190E94FB1A892B75
:1036B00031F0DF91CF911F910F91FF90089580E736
:1036C00099E00E94221915B885B1816485B92D9AB7
:1036D00085B1837E85B91AE1812F8A95F1F7299A00
:1036E00080E28A95F1F72E9880E29EE4FC01319702
:1036F000F1F72E9AFC013197F1F729980197F1F72C
:1037000015B88CE699E00E9422198BE899E00E9496
:10371000221915B812B81A95F1F785B1816485B9E7
:103720002D9885B18C6185B985E08A95F1F7299A44
:1037300080E58A95F1F7C0E0D0E005E04AE1F42E9B
:1037400012E0CE018F779070892B09F47EC0FE01C4
:10375000E95EF94F808182B9802F8A95F1F72E9822
:103760008F2D8A95F1F72E9A3099FECF309BFECFA0
:103770002F9A812F8A95F1F72F98812F8A95F1F74B
:10378000802F8A95F1F7219688E0C030D807C9F6D6
:1037900080E29EE4FC013197F1F729980197F1F757
:1037A00015B812B883E899E00E9422198EEE98E0CD
:1037B0000E94221911B815B88AE18A95F1F785B1EE
:1037C000816485B985B18F7C85B985B18C6085B9F7
:1037D00085E08A95F1F7C0E0D0E012E005E017C07F
:1037E00080B1FE01E95EF94F9081891701F52F9AAA
:1037F000812F8A95F1F72F98812F8A95F1F7802FE5
:103800008A95F1F7219688E0C030D80719F1CE01EA
:103810008F779070892B21F78CEE98E00E94221907
:1038200080B1FE01E95EF94F9081891701F387EDC0
:1038300098E00E94221915B88FEF81B912B8DF9174
:10384000CF911F910F91FF90089589E899E00E9410
:1038500022197DCF15B88FEF81B912B882ED98E0AB
:103860000E94221926CF4F925F926F927F928F9281
:103870009F92AF92BF92CF92DF92EF92FF920F93FF
:103880001F93CF93DF930A98119A85E0982F9A950A
:10389000F1F71198982F9A95F1F7119A982F9A9518
:1038A000F1F720B1982F9A95F1F71198982F9A95E2
:1038B000F1F7119A8A95F1F70299F9C04424552439
:1038C00085E0982F9A95F1F71198982F9A95F1F72E
:1038D000119A982F9A95F1F790B1482F4A95F1F7E0
:1038E0001198482F4A95F1F7119A8A95F1F70299A4
:1038F00001C16624772485E0482F4A95F1F7119895
:10390000482F4A95F1F7119A8A95F1F70299EEC07E
:103910008824992485E0482F4A95F1F71198482F7B
:103920004A95F1F7119A8A95F1F70299DBC0AA241A
:10393000BB2485E0482F4A95F1F71198482F4A9506
:10394000F1F7119A8A95F1F70299C8C0CC24DD24C9
:1039500085E0482F4A95F1F71198482F4A95F1F7DD
:10396000119A8A95F1F70299B5C0EE24FF2485E0FB
:10397000482F4A95F1F71198482F4A95F1F7119A77
:103980008A95F1F70299A3C000E010E085E0482F86
:103990004A95F1F71198482F4A95F1F7119A8A95AF
:1039A000F1F7029991C0C0E0D0E085E0482F4A9538
:1039B000F1F71198482F4A95F1F7119A8A95F1F786
:1039C00002997FC0A0E0B0E085E0482F4A95F1F76A
:1039D0001198482F4A95F1F7119A8A95F1F70299B3
:1039E0006DC0E0E0F0E085E0482F4A95F1F71198CE
:1039F000482F4A95F1F7119A8A95F1F702995BC021
:103A000060E070E085E0482F4A95F1F71198482F63
:103A10004A95F1F7119A8A95F1F702996FC040E043
:103A200050E030E036952795369527952170307017
:103A3000892F90E084709070282B392B2429352908
:103A400026293729282939292A293B292C293D29A2
:103A50002E293F29202B312B2C2B3D2B2A2B3B2B86
:103A60002E2B3F2B262B372B85E0982F9A95F1F79D
:103A70001198982F9A95F1F7119A8A95F1F7119864
:103A800082E08A95F1F7242B352BC901DF91CF9184
:103A90001F910F91FF90EF90DF90CF90BF90AF906C
:103AA0009F908F907F906F905F904F900895E2E08D
:103AB0004E2E512C05CF60E070E1A4CFE0E0F8E09D
:103AC00092CFA0E0B4E080CFC0E0D2E06ECF00E0C3
:103AD00011E05CCF30E8E32EF12C49CF40E4C42E56
:103AE000D12C36CF50E2A52EB12C23CF60E1862E0B
:103AF000912C10CF78E0672E712CFDCE40E050E283
:103B000090CFAC010A9A119A129885E0282F2A9535
:103B1000F1F71198282F2A95F1F7119A8A95F1F764
:103B200040FFE5C082B1846082B985E0282F2A95E4
:103B3000F1F71198282F2A95F1F7119A8A95F1F744
:103B400041FFF9C082B1846082B985E0282F2A95AF
:103B5000F1F71198282F2A95F1F7119A8A95F1F724
:103B600042FFE6C082B1846082B985E0282F2A95A1
:103B7000F1F71198282F2A95F1F7119A8A95F1F704
:103B800043FFD3C082B1846082B985E0282F2A9593
:103B9000F1F71198282F2A95F1F7119A8A95F1F7E4
:103BA00044FFC0C082B1846082B985E0282F2A9585
:103BB000F1F71198282F2A95F1F7119A8A95F1F7C4
:103BC00045FFADC082B1846082B985E0282F2A9577
:103BD000F1F71198282F2A95F1F7119A8A95F1F7A4
:103BE00046FF9AC082B1846082B985E0282F2A9569
:103BF000F1F71198282F2A95F1F7119A8A95F1F784
:103C000047FF87C082B1846082B985E0282F2A955A
:103C1000F1F71198282F2A95F1F7119A8A95F1F763
:103C200050FF74C082B1846082B985E0282F2A9544
:103C3000F1F71198282F2A95F1F7119A8A95F1F743
:103C400051FF61C082B1846082B985E0282F2A9536
:103C5000F1F71198282F2A95F1F7119A8A95F1F723
:103C600052FF4EC082B1846082B985E0282F2A9528
:103C7000F1F71198282F2A95F1F7119A8A95F1F703
:103C800053FF3BC082B1846082B985E0282F2A951A
:103C9000F1F71198282F2A95F1F7119A8A95F1F7E3
:103CA00054FF28C082B1846082B985E0282F2A950C
:103CB000F1F71198282F2A95F1F7119A8A95F1F7C3
:103CC00055FD3CC082B18B7F82B985E0982F9A95D3
:103CD000F1F71198982F9A95F1F7119A8A95F1F7C3
:103CE000129811980A9882E08A95F1F7089582B1A6
:103CF0008B7F1ACF82B18B7FD7CF82B18B7FC4CF1E
:103D000082B18B7FB1CF82B18B7F9ECF82B18B7F0F
:103D10008BCF82B18B7F78CF82B18B7F65CF82B121
:103D20008B7F52CF82B18B7F3FCF82B18B7F2CCFE5
:103D300082B18B7F19CF82B18B7F06CF82B1846035
:103D4000C3CF6F927F928F929F92AF92BF92CF928A
:103D5000DF92EF92FF920F931F93CF93DF9311980F
:103D60002A982F988DE0982F9A95F1F72A9A982FF4
:103D70009A95F1F72F9A8A95F1F784EB9CE00E94CF
:103D80002219C7E1D6E0AA24BB2415E002E0A0E492
:103D90008A2EAFE19A2EF0E86F2EFEE37F2E44C10B
:103DA000F980EE24970120703F73888190E0282BE2
:103DB000392B8FE32F3F380709F4E8C00A9A119A8C
:103DC0001298812F8A95F1F71198812F8A95F1F732
:103DD000119A812F8A95F1F7129A812F8A95F1F71E
:103DE0001198812F8A95F1F7119A812F8A95F1F711
:103DF0001298812F8A95F1F71198812F8A95F1F702
:103E0000119A812F8A95F1F71298812F8A95F1F7EF
:103E10001198812F8A95F1F7119A812F8A95F1F7E0
:103E20001298812F8A95F1F71198812F8A95F1F7D1
:103E3000119A812F8A95F1F7129811980A98802F7C
:103E40008A95F1F7C9010E94811D80910A068D5360
:103E5000823008F4F4C00A9A119A1298812F8A9538
:103E6000F1F71198812F8A95F1F7119A812F8A9590
:103E7000F1F71298812F8A95F1F71198812F8A9581
:103E8000F1F7119A812F8A95F1F71298812F8A956F
:103E9000F1F71198812F8A95F1F7119A812F8A9560
:103EA000F1F7129A812F8A95F1F71198812F8A954F
:103EB000F1F7119A812F8A95F1F71298812F8A953F
:103EC000F1F71198812F8A95F1F7119A812F8A9530
:103ED000F1F7129811980A98802F8A95F1F7C4018A
:103EE0000197F1F70A9A119A1298812F8A95F1F7A2
:103EF0001198812F8A95F1F7119A812F8A95F1F700
:103F00001298812F8A95F1F71198812F8A95F1F7F0
:103F1000119A812F8A95F1F7129A812F8A95F1F7DC
:103F20001198812F8A95F1F7119A812F8A95F1F7CF
:103F30001298812F8A95F1F71198812F8A95F1F7C0
:103F4000119A812F8A95F1F71298812F8A95F1F7AE
:103F50001198812F8A95F1F7119A812F8A95F1F79F
:103F6000129811980A98802F8A95F1F70E94331CB5
:103F7000D980CC24960120703F73488150E0242BD7
:103F8000352B9F738217930709F0A1C00A9A119AE3
:103F90001298812F8A95F1F71198812F8A95F1F760
:103FA000119A812F8A95F1F7129A812F8A95F1F74C
:103FB0001198812F8A95F1F7119A812F8A95F1F73F
:103FC000129A812F8A95F1F71198812F8A95F1F72E
:103FD000119A812F8A95F1F71298812F8A95F1F71E
:103FE0001198812F8A95F1F7119A812F8A95F1F70F
:103FF0001298812F8A95F1F71198812F8A95F1F700
:10400000119A812F8A95F1F7129811980A98802FAA
:104010008A95F1F70894A11CB11C229680E0A8169D
:1040200084E0B80609F46FC0C5018F719070892BC8
:1040300009F0B6CE82EB9CE00E942219B1CE0A9A1A
:10404000119A1298812F8A95F1F71198812F8A95EC
:10405000F1F7119A812F8A95F1F71298812F8A959D
:10406000F1F71198812F8A95F1F7119A812F8A958E
:10407000F1F71298812F8A95F1F71198812F8A957F
:10408000F1F7119A812F8A95F1F7129A812F8A956B
:10409000F1F71198812F8A95F1F7119A812F8A955E
:1040A000F1F7129A812F8A95F1F71198812F8A954D
:1040B000F1F7119A812F8A95F1F7129811980A98C1
:1040C000802F8A95F1F7C3010197F1F70BCF8AE8AA
:1040D0009CE00E94221989E69CE00E9422192F98F8
:1040E0002A982FEF3FEFC901DF91CF911F910F91D8
:1040F000FF90EF90DF90CF90BF90AF909F908F9008
:104100007F906F9008952F982A9820E030E0EBCFB1
:10411000CF92DF92EF92FF920F931F93CF93DF9393
:1041200011982A982F988DE0982F9A95F1F72A9A4E
:10413000982F9A95F1F72F9A8A95F1F789E49CE0E8
:104140000E942219C7E1DEE015E002E080E4E82EDB
:104150008FE1F82EB0E8CB2EBEE3DB2EDEC00A9A4C
:10416000119A1298812F8A95F1F71198812F8A95CB
:10417000F1F7119A812F8A95F1F71298812F8A957C
:10418000F1F71198812F8A95F1F7119A812F8A956D
:10419000F1F71298812F8A95F1F71198812F8A955E
:1041A000F1F7119A812F8A95F1F7129A812F8A954A
:1041B000F1F71198812F8A95F1F7119A812F8A953D
:1041C000F1F71298812F8A95F1F71198812F8A952E
:1041D000F1F7119A812F8A95F1F7129811980A98A0
:1041E000802F8A95F1F7C7010197F1F70A9A119A82
:1041F000129A812F8A95F1F71198812F8A95F1F7FC
:10420000119A812F8A95F1F71298812F8A95F1F7EB
:104210001198812F8A95F1F7119A812F8A95F1F7DC
:10422000129A812F8A95F1F71198812F8A95F1F7CB
:10423000119A812F8A95F1F71298812F8A95F1F7BB
:104240001198812F8A95F1F7119A812F8A95F1F7AC
:104250001298812F8A95F1F71198812F8A95F1F79D
:10426000119A812F8A95F1F7129811980A98802F48
:104270008A95F1F70E94331C90E0288130E0821784
:10428000930709F0E3C00A9A119A1298812F8A9530
:10429000F1F71198812F8A95F1F7119A812F8A955C
:1042A000F1F7129A812F8A95F1F71198812F8A954B
:1042B000F1F7119A812F8A95F1F7129A812F8A9539
:1042C000F1F71198812F8A95F1F7119A812F8A952C
:1042D000F1F71298812F8A95F1F71198812F8A951D
:1042E000F1F7119A812F8A95F1F71298812F8A950B
:1042F000F1F71198812F8A95F1F7119A812F8A95FC
:10430000F1F7129811980A98802F8A95F1F7219663
:104310008EE0C739D80709F4ABC088818F3F09F414
:10432000B2CF0A9A119A129A912F9A95F1F7119891
:10433000912F9A95F1F7119A912F9A95F1F7129A78
:10434000912F9A95F1F71198912F9A95F1F7119A6B
:10435000912F9A95F1F71298912F9A95F1F711985C
:10436000912F9A95F1F7119A912F9A95F1F712984A
:10437000912F9A95F1F71198912F9A95F1F7119A3B
:10438000912F9A95F1F71298912F9A95F1F711982C
:10439000912F9A95F1F7119A912F9A95F1F712981A
:1043A00011980A98902F9A95F1F790E00E94811D3C
:1043B00080910A068D53823008F0D1CE0A9A119A64
:1043C0001298812F8A95F1F71198812F8A95F1F72C
:1043D000119A812F8A95F1F71298812F8A95F1F71A
:1043E0001198812F8A95F1F7119A812F8A95F1F70B
:1043F0001298812F8A95F1F71198812F8A95F1F7FC
:10440000119A812F8A95F1F7129A812F8A95F1F7E7
:104410001198812F8A95F1F7119A812F8A95F1F7DA
:10442000129A812F8A95F1F71198812F8A95F1F7C9
:10443000119A812F8A95F1F7129811980A98802F76
:104440008A95F1F7C6010197F1F7D0CE8CE19CE097
:104450000E9422192F982A982FEF3FEFC901DF9170
:10446000CF911F910F91FF90EF90DF90CF90089523
:104470002F982A9820E030E0F1CF8F929F92AF9250
:10448000BF92CF92DF92EF92FF920F931F93DF9331
:10449000CF93CDB7DEB72A970FB6F894DEBF0FBE25
:1044A000CDBF11982A982F988DE0982F9A95F1F703
:1044B0002A9A982F9A95F1F72F9A8A95F1F70A9AE6
:1044C000119A129885E0982F9A95F1F71198982FE4
:1044D0009A95F1F7119A982F9A95F1F7129A982FC9
:1044E0009A95F1F71198982F9A95F1F7119A982FBC
:1044F0009A95F1F71298982F9A95F1F71198982FAD
:104500009A95F1F7119A982F9A95F1F71298982F9A
:104510009A95F1F71198982F9A95F1F7119A982F8B
:104520009A95F1F71298982F9A95F1F71198982F7C
:104530009A95F1F7119A8A95F1F7129811980A98BD
:1045400082E08A95F1F780E090E00E94811DEE24E0
:10455000FF245E010894A11CB11C71E1872E72E05A
:10456000972E05E062E0D62E98C00A9A119A12980A
:10457000802F8A95F1F71198802F8A95F1F7119A7B
:10458000802F8A95F1F71298802F8A95F1F711986C
:10459000802F8A95F1F7119A802F8A95F1F7129A58
:1045A000802F8A95F1F71198802F8A95F1F7119A4B
:1045B000802F8A95F1F71298802F8A95F1F711983C
:1045C000802F8A95F1F7119A802F8A95F1F712982A
:1045D000802F8A95F1F71198802F8A95F1F7119A1B
:1045E000802F8A95F1F7129811980A988D2D8A9547
:1045F000F1F70E94331C192F0E944119812F0E944C
:1046000041190A9A119A1298802F8A95F1F71198F8
:10461000802F8A95F1F7119A802F8A95F1F7129AD7
:10462000802F8A95F1F71198802F8A95F1F7119ACA
:10463000802F8A95F1F7129A802F8A95F1F71198B9
:10464000802F8A95F1F7119A802F8A95F1F71298A9
:10465000802F8A95F1F71198802F8A95F1F7119A9A
:10466000802F8A95F1F71298802F8A95F1F711988B
:10467000802F8A95F1F7119A802F8A95F1F7129879
:1046800011980A988D2D8A95F1F70894E11CF11C78
:1046900090E0E91694E0F90659F1C7018F70907027
:1046A000892B09F062CF8EEF99E00E94221900D089
:1046B00000D000D0EDB7FEB73196ADB7BEB71296B9
:1046C000BC92AE92119793828282C701880F991F84
:1046D000958384830E9455398DB79EB706960FB691
:1046E000F8949EBF0FBE8DBFC5010E9409193DCF32
:1046F0002F982A9811982A982F988DE0982F9A959C
:10470000F1F72A9A982F9A95F1F72F9A8A95F1F74F
:1047100085EF99E00E942219EE24FF245E0108949F
:10472000A11CB11C41E1842E42E0942E15E002E070
:1047300097C00A9A119A129A35E0D32E812F8A9542
:10474000F1F71198812F8A95F1F7119A812F8A95A7
:10475000F1F71298812F8A95F1F71198812F8A9598
:10476000F1F7119A812F8A95F1F7129A812F8A9584
:10477000F1F71198812F8A95F1F7119A812F8A9577
:10478000F1F71298812F8A95F1F71198812F8A9568
:10479000F1F7119A812F8A95F1F71298812F8A9556
:1047A000F1F71198812F8A95F1F7119A812F8A9547
:1047B000F1F7129811980A9822E0C22E802F8A955C
:1047C000F1F70E94331C0E9441190A9A119A12981B
:1047D000812F8A95F1F71198812F8A95F1F7119A17
:1047E000812F8A95F1F7129A812F8A95F1F7119806
:1047F000812F8A95F1F7119A812F8A95F1F7129AF4
:10480000812F8A95F1F71198812F8A95F1F7119AE6
:10481000812F8A95F1F71298812F8A95F1F71198D7
:10482000812F8A95F1F7119A812F8A95F1F71298C5
:10483000812F8A95F1F71198812F8A95F1F7119AB6
:10484000812F8A95F1F7129811980A98802F8A95EE
:10485000F1F70894E11CF11C90E8E916F10441F12C
:10486000C7018F719070892B09F063CF83EF99E0B6
:104870000E94221900D000D000D0EDB7FEB73196CB
:10488000ADB7BEB71296BC92AE9211979382828258
:10489000F582E4820E9455398DB79EB706960FB611
:1048A000F8949EBF0FBE8DBFC5010E94091941CF6C
:1048B0002F982A9811982A982F988DE0982F9A95DA
:1048C000F1F72A9A982F9A95F1F72F9A8A95F1F78E
:1048D0000A9A119A129805E08D2D8A95F1F7119890
:1048E0008D2D8A95F1F7119A8D2D8A95F1F71298F1
:1048F0008D2D8A95F1F711988D2D8A95F1F7119AE2
:104900008D2D8A95F1F712988D2D8A95F1F71198D2
:104910008D2D8A95F1F7119A8D2D8A95F1F71298C0
:104920008D2D8A95F1F711988D2D8A95F1F7119AB1
:104930008D2D8A95F1F712988D2D8A95F1F71198A2
:104940008D2D8A95F1F7119A8D2D8A95F1F7129890
:1049500011980A9892E0F92E8C2D8A95F1F78FEF35
:104960009FE30E94811D86EE99E00E9422190A9A17
:10497000119A12988D2D8A95F1F711988D2D8A959F
:10498000F1F7119A8D2D8A95F1F712988D2D8A9550
:10499000F1F711988D2D8A95F1F7119A8D2D8A9541
:1049A000F1F7129A8D2D8A95F1F711988D2D8A9530
:1049B000F1F7119A8D2D8A95F1F712988D2D8A9520
:1049C000F1F711988D2D8A95F1F7119A8D2D8A9511
:1049D000F1F712988D2D8A95F1F711988D2D8A9502
:1049E000F1F7119A8D2D8A95F1F7129811980A987E
:1049F0008C2D8A95F1F70E94331C192F0E944119C2
:104A0000812F0E9441190A9A119A12988D2D8A9528
:104A1000F1F711988D2D8A95F1F7119A8D2D8A95C0
:104A2000F1F7129A8D2D8A95F1F711988D2D8A95AF
:104A3000F1F7119A8D2D8A95F1F7129A8D2D8A959D
:104A4000F1F711988D2D8A95F1F7119A8D2D8A9590
:104A5000F1F712988D2D8A95F1F711988D2D8A9581
:104A6000F1F7119A8D2D8A95F1F712988D2D8A956F
:104A7000F1F711988D2D8A95F1F7119A8D2D8A9560
:104A8000F1F7129811980A988C2D8A95F1F70A9AE5
:104A9000119A12988D2D8A95F1F711988D2D8A957E
:104AA000F1F7119A8D2D8A95F1F712988D2D8A952F
:104AB000F1F711988D2D8A95F1F7119A8D2D8A9520
:104AC000F1F7129A8D2D8A95F1F711988D2D8A950F
:104AD000F1F7119A8D2D8A95F1F712988D2D8A95FF
:104AE000F1F711988D2D8A95F1F7119A8D2D8A95F0
:104AF000F1F712988D2D8A95F1F711988D2D8A95E1
:104B0000F1F7119A8D2D8A95F1F7129811980A985C
:104B10008C2D8A95F1F70E94331C192F0E944119A0
:104B2000812F0E9441190A9A119A12988D2D8A9507
:104B3000F1F711988D2D8A95F1F7119A8D2D8A959F
:104B4000F1F7129A8D2D8A95F1F711988D2D8A958E
:104B5000F1F7119A8D2D8A95F1F7129A8D2D8A957C
:104B6000F1F711988D2D8A95F1F7119A8D2D8A956F
:104B7000F1F712988D2D8A95F1F711988D2D8A9560
:104B8000F1F7119A8D2D8A95F1F712988D2D8A954E
:104B9000F1F711988D2D8A95F1F7119A8D2D8A953F
:104BA000F1F7129811980A988C2D8A95F1F70A9AC4
:104BB000119A12988D2D8A95F1F711988D2D8A955D
:104BC000F1F7119A8D2D8A95F1F712988D2D8A950E
:104BD000F1F711988D2D8A95F1F7119A8D2D8A95FF
:104BE000F1F7129A8D2D8A95F1F711988D2D8A95EE
:104BF000F1F7119A8D2D8A95F1F712988D2D8A95DE
:104C0000F1F711988D2D8A95F1F7119A8D2D8A95CE
:104C1000F1F712988D2D8A95F1F711988D2D8A95BF
:104C2000F1F7119A8D2D8A95F1F7129811980A983B
:104C30008C2D8A95F1F70E94331C192F0E9441197F
:104C4000812F0E9441190A9A119A12988D2D8A95E6
:104C5000F1F711988D2D8A95F1F7119A8D2D8A957E
:104C6000F1F7129A8D2D8A95F1F711988D2D8A956D
:104C7000F1F7119A8D2D8A95F1F7129A8D2D8A955B
:104C8000F1F711988D2D8A95F1F7119A8D2D8A954E
:104C9000F1F712988D2D8A95F1F711988D2D8A953F
:104CA000F1F7119A8D2D8A95F1F712988D2D8A952D
:104CB000F1F711988D2D8A95F1F7119A8D2D8A951E
:104CC000F1F7129811980A988C2D8A95F1F70A9AA3
:104CD000119A12988D2D8A95F1F711988D2D8A953C
:104CE000F1F7119A8D2D8A95F1F712988D2D8A95ED
:104CF000F1F711988D2D8A95F1F7119A8D2D8A95DE
:104D0000F1F7129A8D2D8A95F1F711988D2D8A95CC
:104D1000F1F7119A8D2D8A95F1F712988D2D8A95BC
:104D2000F1F711988D2D8A95F1F7119A8D2D8A95AD
:104D3000F1F712988D2D8A95F1F711988D2D8A959E
:104D4000F1F7119A8D2D8A95F1F7129811980A981A
:104D50008C2D8A95F1F70E94331C192F0E9441195E
:104D6000812F0E9441190A9A119A12988D2D8A95C5
:104D7000F1F711988D2D8A95F1F7119A8D2D8A955D
:104D8000F1F7129A8D2D8A95F1F711988D2D8A954C
:104D9000F1F7119A8D2D8A95F1F7129A8D2D8A953A
:104DA000F1F711988D2D8A95F1F7119A8D2D8A952D
:104DB000F1F712988D2D8A95F1F711988D2D8A951E
:104DC000F1F7119A8D2D8A95F1F712988D2D8A950C
:104DD000F1F711988D2D8A95F1F7119A8D2D8A95FD
:104DE000F1F7129811980A988C2D8A95F1F70A9A82
:104DF000119A12988D2D8A95F1F711988D2D8A951B
:104E0000F1F7119A8D2D8A95F1F7129A8D2D8A95C9
:104E1000F1F711988D2D8A95F1F7119A8D2D8A95BC
:104E2000F1F7129A8D2D8A95F1F711988D2D8A95AB
:104E3000F1F7119A8D2D8A95F1F712988D2D8A959B
:104E4000F1F711988D2D8A95F1F7119A8D2D8A958C
:104E5000F1F712988D2D8A95F1F711988D2D8A957D
:104E6000F1F7119A8D2D8A95F1F7129811980A98F9
:104E70008C2D8A95F1F70A9A119A12988D2D8A95A0
:104E8000F1F711988D2D8A95F1F7119A8D2D8A954C
:104E9000F1F7129A802F8A95F1F71198802F8A9551
:104EA000F1F7119A802F8A95F1F7129A802F8A953F
:104EB000F1F71198802F8A95F1F7119A802F8A9532
:104EC000F1F71298802F8A95F1F71198802F8A9523
:104ED000F1F7119A802F8A95F1F71298802F8A9511
:104EE000F1F71198802F8A95F1F7119A802F8A9502
:104EF000F1F7129811980A988F2D8A95F1F70A9A6E
:104F0000119A1298802F8A95F1F71198802F8A951F
:104F1000F1F7119A802F8A95F1F7129A802F8A95CE
:104F2000F1F71198802F8A95F1F7119A802F8A95C1
:104F3000F1F7129A802F8A95F1F71198802F8A95B0
:104F4000F1F7119A802F8A95F1F71298802F8A95A0
:104F5000F1F71198802F8A95F1F7119A802F8A9591
:104F6000F1F71298802F8A95F1F71198802F8A9582
:104F7000F1F7119A802F8A95F1F7129811980A98F3
:104F80008F2D8A95F1F785ED99E00E9422190A9AF2
:104F9000119A1298802F8A95F1F71198802F8A958F
:104FA000F1F7119A802F8A95F1F71298802F8A9540
:104FB000F1F71198802F8A95F1F7119A802F8A9531
:104FC000F1F7129A802F8A95F1F71198802F8A9520
:104FD000F1F7119A802F8A95F1F71298802F8A9510
:104FE000F1F71198802F8A95F1F7119A802F8A9501
:104FF000F1F71298802F8A95F1F71198802F8A95F2
:10500000F1F7119A0A95F1F7129811980A98FA9403
:10501000F1F70E94331C192F0E944119812F0E9421
:1050200041192F982A982A960FB6F894DEBF0FBE22
:10503000CDBFCF91DF911F910F91FF90EF90DF9047
:10504000CF90BF90AF909F908F9008950F931F9334
:10505000DF93CF930F92CDB7DEB711982A982F9890
:105060008DE0982F9A95F1F72A9A982F9A95F1F753
:105070002F9A8A95F1F70A9A119A129815E0812FC2
:105080008A95F1F71198812F8A95F1F7119A812F5E
:105090008A95F1F71298812F8A95F1F71198812F4F
:1050A0008A95F1F7119A812F8A95F1F71298812F3D
:1050B0008A95F1F71198812F8A95F1F7119A812F2E
:1050C0008A95F1F71298812F8A95F1F71198812F1F
:1050D0008A95F1F7119A812F8A95F1F71298812F0D
:1050E0008A95F1F71198812F8A95F1F7119A812FFE
:1050F0008A95F1F7129811980A9802E0802F8A9504
:10510000F1F780E090E00E94811D0A9A119A1298AE
:10511000812F8A95F1F71198812F8A95F1F7119ACD
:10512000812F8A95F1F7129A812F8A95F1F71198BC
:10513000812F8A95F1F7119A812F8A95F1F7129AAA
:10514000812F8A95F1F71198812F8A95F1F7119A9D
:10515000812F8A95F1F71298812F8A95F1F711988E
:10516000812F8A95F1F7119A812F8A95F1F712987C
:10517000812F8A95F1F71198812F8A95F1F7119A6D
:10518000812F8A95F1F7129811980A98802F8A95A5
:10519000F1F70A9A119A1298812F8A95F1F71198CE
:1051A000812F8A95F1F7119A812F8A95F1F7129A3A
:1051B000812F8A95F1F71198812F8A95F1F7119A2D
:1051C000812F8A95F1F7129A812F8A95F1F711981C
:1051D000812F8A95F1F7119A812F8A95F1F712980C
:1051E000812F8A95F1F71198812F8A95F1F7119AFD
:1051F000812F8A95F1F71298812F8A95F1F71198EE
:10520000812F8A95F1F7119A812F8A95F1F71298DB
:1052100011980A98802F8A95F1F70A9A119A129894
:10522000812F8A95F1F71198812F8A95F1F7119ABC
:10523000812F8A95F1F7129A812F8A95F1F71198AB
:10524000812F8A95F1F7119A812F8A95F1F7129A99
:10525000812F8A95F1F71198812F8A95F1F7119A8C
:10526000812F8A95F1F71298812F8A95F1F711987D
:10527000812F8A95F1F7119A812F8A95F1F712986B
:10528000812F8A95F1F71198812F8A95F1F7119A5C
:10529000812F8A95F1F7129811980A98802F8A9594
:1052A000F1F70A9A119A1298812F8A95F1F71198BD
:1052B000812F8A95F1F7119A812F8A95F1F7129A29
:1052C000812F8A95F1F71198812F8A95F1F7119A1C
:1052D000812F8A95F1F7129A812F8A95F1F711980B
:1052E000812F8A95F1F7119A812F8A95F1F71298FB
:1052F000812F8A95F1F71198812F8A95F1F7119AEC
:10530000812F8A95F1F71298812F8A95F1F71198DC
:10531000812F8A95F1F7119A812F8A95F1F71298CA
:1053200011980A98802F8A95F1F70A9A119A129883
:10533000812F8A95F1F71198812F8A95F1F7119AAB
:10534000812F8A95F1F7129A812F8A95F1F711989A
:10535000812F8A95F1F7119A812F8A95F1F7129A88
:10536000812F8A95F1F71198812F8A95F1F7119A7B
:10537000812F8A95F1F71298812F8A95F1F711986C
:10538000812F8A95F1F7119A812F8A95F1F712985A
:10539000812F8A95F1F71198812F8A95F1F7119A4B
:1053A000812F8A95F1F7129811980A98802F8A9583
:1053B000F1F70A9A119A1298812F8A95F1F71198AC
:1053C000812F8A95F1F7119A812F8A95F1F7129A18
:1053D000812F8A95F1F71198812F8A95F1F7119A0B
:1053E000812F8A95F1F7129A812F8A95F1F71198FA
:1053F000812F8A95F1F7119A812F8A95F1F71298EA
:10540000812F8A95F1F71198812F8A95F1F7119ADA
:10541000812F8A95F1F71298812F8A95F1F71198CB
:10542000812F8A95F1F7119A812F8A95F1F71298B9
:1054300011980A98802F8A95F1F70A9A119A129872
:10544000812F8A95F1F71198812F8A95F1F7119A9A
:10545000812F8A95F1F71298812F8A95F1F711988B
:10546000812F8A95F1F7119A812F8A95F1F7129A77
:10547000812F8A95F1F71198812F8A95F1F7119A6A
:10548000812F8A95F1F71298812F8A95F1F711985B
:10549000812F8A95F1F7119A812F8A95F1F7129849
:1054A000812F8A95F1F71198812F8A95F1F7119A3A
:1054B0001A95F1F7129811980A980A95F1F70E9437
:1054C000331C8C0116950795129502950F700127D4
:1054D0001F70012710700238110509F46BC00338E2
:1054E0001105D0F00338110509F446C0083811053C
:1054F00041F180E09AE00E94221980E00E94411967
:10550000802F09830E9441199981892F0F90CF9193
:10551000DF911F910F9108950D331105E1F10E33C5
:10552000110539F78FE19AE00E9422198EE38093EA
:105530000A069EE3892F0F90CF91DF911F910F9163
:1055400008958DE29BE00E9422198CED9AE00E9462
:1055500022198EEB9AE00E94221981E79AE00E94BC
:10556000221988E880930A0698E8892F0F90CF9136
:10557000DF911F910F91089587E49AE00E9422190C
:1055800083E880930A0693E8892F0F90CF91DF91EB
:105590001F910F91089583E39AE00E9422198DE3F1
:1055A00080930A069DE3892F0F90CF91DF911F9181
:1055B0000F9108958CE59AE00E94221982E8809369
:1055C0000A0692E8892F0F90CF91DF911F910F91DA
:1055D00008952F923F925F926F927F928F929F9247
:1055E000AF92BF92CF92DF92EF92FF920F931F93F1
:1055F000CF93DF9385EF9BE00E94221911982A98A0
:105600002F988DE0982F9A95F1F72A9A982F9A95CE
:10561000F1F72F9A8A95F1F70A9A119A129885E074
:10562000982F9A95F1F71198982F9A95F1F7119A6A
:10563000982F9A95F1F71298982F9A95F1F711985B
:10564000982F9A95F1F7119A982F9A95F1F7129849
:10565000982F9A95F1F71198982F9A95F1F7119A3A
:10566000982F9A95F1F71298982F9A95F1F711982B
:10567000982F9A95F1F7119A982F9A95F1F7129819
:10568000982F9A95F1F71198982F9A95F1F7119A0A
:105690008A95F1F7129811980A9882E08A95F1F7A5
:1056A0008FEF9FE30E94811DB7E9EB2EBEE0FB2E3A
:1056B0000CEF8824992415E0A2E05A2EF0E42F2E56
:1056C000FFE13F2EECC00A9A119A1298812F8A9519
:1056D000F1F71198812F8A95F1F7119A812F8A9508
:1056E000F1F71298812F8A95F1F71198812F8A95F9
:1056F000F1F7119A812F8A95F1F71298812F8A95E7
:10570000F1F71198812F8A95F1F7119A812F8A95D7
:10571000F1F7129A812F8A95F1F71198812F8A95C6
:10572000F1F7119A812F8A95F1F71298812F8A95B6
:10573000F1F71198812F8A95F1F7119A812F8A95A7
:10574000F1F7129811980A98852D8A95F1F7C10101
:105750000197F1F70A9A119A1298812F8A95F1F719
:105760001198812F8A95F1F7119A812F8A95F1F777
:105770001298812F8A95F1F71198812F8A95F1F768
:10578000119A812F8A95F1F7129A812F8A95F1F754
:105790001198812F8A95F1F7119A812F8A95F1F747
:1057A0001298812F8A95F1F71198812F8A95F1F738
:1057B000119A812F8A95F1F71298812F8A95F1F726
:1057C0001198812F8A95F1F7119A812F8A95F1F717
:1057D000129811980A98852D8A95F1F70E94331C2A
:1057E000EC01F701B180AA24C50180709F7320816C
:1057F00030E0822B932B9E013F732817390709F065
:1058000011C10A9A119A1298812F8A95F1F711986D
:10581000812F8A95F1F7119A812F8A95F1F7129AC3
:10582000812F8A95F1F71198812F8A95F1F7119AB6
:10583000812F8A95F1F7129A812F8A95F1F71198A5
:10584000812F8A95F1F7119A812F8A95F1F7129895
:10585000812F8A95F1F71198812F8A95F1F7119A86
:10586000812F8A95F1F71298812F8A95F1F7119877
:10587000812F8A95F1F7119A812F8A95F1F7129865
:1058800011980A98852D8A95F1F70F5F82E090E0D4
:10589000880E991EE80EF91E043009F4ACC00330DE
:1058A00008F4AFCF34010894611C711CF701D1805A
:1058B000CC24960120703F73808190E0282B392BF7
:1058C000FFE32F3F3F0709F49CCF0A9A119A1298E1
:1058D000812F8A95F1F71198812F8A95F1F7119A06
:1058E000812F8A95F1F7129A812F8A95F1F71198F5
:1058F000812F8A95F1F7119A812F8A95F1F71298E5
:10590000812F8A95F1F71198812F8A95F1F7119AD5
:10591000812F8A95F1F71298812F8A95F1F71198C6
:10592000812F8A95F1F7119A812F8A95F1F71298B4
:10593000812F8A95F1F71198812F8A95F1F7119AA5
:10594000812F8A95F1F7129811980A98852D8A95DA
:10595000F1F7C9010E94811D80910A068D538230A2
:1059600008F0B1CE0A9A119A1298812F8A95F1F710
:105970001198812F8A95F1F7119A812F8A95F1F765
:105980001298812F8A95F1F71198812F8A95F1F756
:10599000119A812F8A95F1F71298812F8A95F1F744
:1059A0001198812F8A95F1F7119A812F8A95F1F735
:1059B000129A812F8A95F1F71198812F8A95F1F724
:1059C000119A812F8A95F1F71298812F8A95F1F714
:1059D0001198812F8A95F1F7119A812F8A95F1F705
:1059E000129811980A98852D8A95F1F780E995E625
:1059F0000197F1F7AFCE2F982A9820E030E0C90147
:105A0000DF91CF911F910F91FF90EF90DF90CF909A
:105A1000BF90AF909F908F907F906F905F903F90DE
:105A20002F9008958FEB9BE00E94221986EB9BE05C
:105A30000E94221987E99EE0680E791EF301808199
:105A40000E94411987E99EE0880E991EF401808129
:105A50000E9441198DEA9BE00E9422198D2F0E941D
:105A600041198C2F0E9441198EE69BE00E94221959
:105A700082E49BE00E9422192F982A982FEF3FEF93
:105A8000BECF0F931F938CE999E00E9422191198C1
:105A90002A982F988DE0982F9A95F1F72A9A982FA7
:105AA0009A95F1F72F9A8A95F1F780910A068D530E
:105AB000823008F495C00A9A119A129815E0812F45
:105AC0008A95F1F71198812F8A95F1F7119A812F14
:105AD0008A95F1F71298812F8A95F1F71198812F05
:105AE0008A95F1F7119A812F8A95F1F71298812FF3
:105AF0008A95F1F71198812F8A95F1F7119A812FE4
:105B00008A95F1F71298812F8A95F1F71198812FD4
:105B10008A95F1F7119A812F8A95F1F71298812FC2
:105B20008A95F1F71198812F8A95F1F7119A812FB3
:105B30008A95F1F7129811980A9802E0802F8A95B9
:105B4000F1F78FEF9FE30E94811D0A9A119A129A32
:105B5000812F8A95F1F71198812F8A95F1F7119A83
:105B6000812F8A95F1F71298812F8A95F1F7119874
:105B7000812F8A95F1F7119A812F8A95F1F7129862
:105B8000812F8A95F1F71198812F8A95F1F7119A53
:105B9000812F8A95F1F7129A812F8A95F1F7119842
:105BA000812F8A95F1F7119A812F8A95F1F7129832
:105BB000812F8A95F1F71198812F8A95F1F7119A23
:105BC0001A95F1F7129811980A980A95F1F780EE54
:105BD0009EE20197F1F72F982A981F910F9108954F
:105BE0000A9A119A129815E0812F8A95F1F7119867
:105BF000812F8A95F1F7119A812F8A95F1F71298E2
:105C0000812F8A95F1F71198812F8A95F1F7119AD2
:105C1000812F8A95F1F71298812F8A95F1F71198C3
:105C2000812F8A95F1F7119A812F8A95F1F71298B1
:105C3000812F8A95F1F71198812F8A95F1F7119AA2
:105C4000812F8A95F1F71298812F8A95F1F7119893
:105C5000812F8A95F1F7119A812F8A95F1F7129881
:105C600011980A9802E0802F8A95F1F78FEF9FE351
:105C70000E94811D0A9A119A1298812F8A95F1F734
:105C80001198812F8A95F1F7119A812F8A95F1F752
:105C9000129A812F8A95F1F71198812F8A95F1F741
:105CA000119A812F8A95F1F7129A812F8A95F1F72F
:105CB0001198812F8A95F1F7119A812F8A95F1F722
:105CC0001298812F8A95F1F71198812F8A95F1F713
:105CD000119A812F8A95F1F71298812F8A95F1F701
:105CE0001198812F8A95F1F7119A812F8A95F1F7F2
:105CF000129811980A98802F8A95F1F70A9A119AAA
:105D00001298812F8A95F1F71198812F8A95F1F7D2
:105D1000119A812F8A95F1F7129A812F8A95F1F7BE
:105D20001198812F8A95F1F7119A812F8A95F1F7B1
:105D3000129A812F8A95F1F71198812F8A95F1F7A0
:105D4000119A812F8A95F1F71298812F8A95F1F790
:105D50001198812F8A95F1F7119A812F8A95F1F781
:105D60001298812F8A95F1F71198812F8A95F1F772
:105D7000119A812F8A95F1F7129811980A98802F1D
:105D80008A95F1F70A9A119A1298812F8A95F1F75C
:105D90001198812F8A95F1F7119A812F8A95F1F741
:105DA000129A812F8A95F1F71198812F8A95F1F730
:105DB000119A812F8A95F1F7129A812F8A95F1F71E
:105DC0001198812F8A95F1F7119A812F8A95F1F711
:105DD0001298812F8A95F1F71198812F8A95F1F702
:105DE000119A812F8A95F1F71298812F8A95F1F7F0
:105DF0001198812F8A95F1F7119A812F8A95F1F7E1
:105E0000129811980A98802F8A95F1F70A9A119A98
:105E10001298812F8A95F1F71198812F8A95F1F7C1
:105E2000119A812F8A95F1F7129A812F8A95F1F7AD
:105E30001198812F8A95F1F7119A812F8A95F1F7A0
:105E4000129A812F8A95F1F71198812F8A95F1F78F
:105E5000119A812F8A95F1F71298812F8A95F1F77F
:105E60001198812F8A95F1F7119A812F8A95F1F770
:105E70001298812F8A95F1F71198812F8A95F1F761
:105E8000119A812F8A95F1F7129811980A98802F0C
:105E90008A95F1F70A9A119A1298812F8A95F1F74B
:105EA0001198812F8A95F1F7119A812F8A95F1F730
:105EB000129A812F8A95F1F71198812F8A95F1F71F
:105EC000119A812F8A95F1F7129A812F8A95F1F70D
:105ED0001198812F8A95F1F7119A812F8A95F1F700
:105EE0001298812F8A95F1F71198812F8A95F1F7F1
:105EF000119A812F8A95F1F71298812F8A95F1F7DF
:105F00001198812F8A95F1F7119A812F8A95F1F7CF
:105F1000129811980A98802F8A95F1F70A9A119A87
:105F20001298812F8A95F1F71198812F8A95F1F7B0
:105F3000119A812F8A95F1F7129A812F8A95F1F79C
:105F40001198812F8A95F1F7119A812F8A95F1F78F
:105F5000129A812F8A95F1F71198812F8A95F1F77E
:105F6000119A812F8A95F1F71298812F8A95F1F76E
:105F70001198812F8A95F1F7119A812F8A95F1F75F
:105F80001298812F8A95F1F71198812F8A95F1F750
:105F9000119A812F8A95F1F7129811980A98802FFB
:105FA0008A95F1F70A9A119A1298812F8A95F1F73A
:105FB0001198812F8A95F1F7119A812F8A95F1F71F
:105FC000129A812F8A95F1F71198812F8A95F1F70E
:105FD000119A812F8A95F1F7129A812F8A95F1F7FC
:105FE0001198812F8A95F1F7119A812F8A95F1F7EF
:105FF0001298812F8A95F1F71198812F8A95F1F7E0
:10600000119A812F8A95F1F71298812F8A95F1F7CD
:106010001198812F8A95F1F7119A812F8A95F1F7BE
:10602000129811980A98802F8A95F1F70A9A119A76
:10603000129A812F8A95F1F71198812F8A95F1F79D
:10604000119A812F8A95F1F71298812F8A95F1F78D
:106050001198812F8A95F1F7119A812F8A95F1F77E
:106060001298812F8A95F1F71198812F8A95F1F76F
:10607000119A812F8A95F1F71298812F8A95F1F75D
:106080001198812F8A95F1F7119A812F8A95F1F74E
:106090001298812F8A95F1F71198812F8A95F1F73F
:1060A000119A812F8A95F1F7129811980A98802FEA
:1060B0008A95F1F70A9A119A129A812F8A95F1F727
:1060C0001198812F8A95F1F7119A812F8A95F1F70E
:1060D000129A812F8A95F1F71198812F8A95F1F7FD
:1060E000119A812F8A95F1F7129A812F8A95F1F7EB
:1060F0001198812F8A95F1F7119A812F8A95F1F7DE
:106100001298812F8A95F1F71198812F8A95F1F7CE
:10611000119A812F8A95F1F71298812F8A95F1F7BC
:106120001198812F8A95F1F7119A812F8A95F1F7AD
:10613000129811980A98802F8A95F1F70A9A119A65
:106140001298812F8A95F1F71198812F8A95F1F78E
:10615000119A812F8A95F1F71298812F8A95F1F77C
:106160001198812F8A95F1F7119A812F8A95F1F76D
:106170001298812F8A95F1F71198812F8A95F1F75E
:10618000119A812F8A95F1F7129A812F8A95F1F74A
:106190001198812F8A95F1F7119A812F8A95F1F73D
:1061A0001298812F8A95F1F71198812F8A95F1F72E
:1061B000119A812F8A95F1F7129811980A98802FD9
:1061C0008A95F1F780E995E60197F1F70A9A119A15
:1061D000129A812F8A95F1F71198812F8A95F1F7FC
:1061E000119A812F8A95F1F71298812F8A95F1F7EC
:1061F0001198812F8A95F1F7119A812F8A95F1F7DD
:106200001298812F8A95F1F71198812F8A95F1F7CD
:10621000119A812F8A95F1F71298812F8A95F1F7BB
:106220001198812F8A95F1F7119A812F8A95F1F7AC
:106230001298812F8A95F1F71198812F8A95F1F79D
:10624000119A812F8A95F1F7129811980A98802F48
:106250008A95F1F70A9A119A129A812F8A95F1F785
:106260001198812F8A95F1F7119A812F8A95F1F76C
:10627000129A812F8A95F1F71198812F8A95F1F75B
:10628000119A812F8A95F1F7129A812F8A95F1F749
:106290001198812F8A95F1F7119A812F8A95F1F73C
:1062A0001298812F8A95F1F71198812F8A95F1F72D
:1062B000119A812F8A95F1F71298812F8A95F1F71B
:1062C0001198812F8A95F1F7119A1A95F1F7129882
:1062D00011980A980A95F1F72F982A981F910F9113
:1062E00008950F931F9311982A982F988DE0982F57
:1062F0009A95F1F72A9A982F9A95F1F72F9A8A95FD
:10630000F1F783EF9CE00E9422190A9A119A1298E1
:1063100015E0812F8A95F1F71198812F8A95F1F771
:10632000119A812F8A95F1F7129A812F8A95F1F7A8
:106330001198812F8A95F1F7119A812F8A95F1F79B
:106340001298812F8A95F1F71198812F8A95F1F78C
:10635000119A812F8A95F1F71298812F8A95F1F77A
:106360001198812F8A95F1F7119A812F8A95F1F76B
:106370001298812F8A95F1F71198812F8A95F1F75C
:10638000119A812F8A95F1F7129811980A9802E0D4
:10639000802F8A95F1F78FEF9FE30E94811D0A9A63
:1063A000119A129A812F8A95F1F71198812F8A9567
:1063B000F1F7119A812F8A95F1F71298812F8A951A
:1063C000F1F71198812F8A95F1F7119A812F8A950B
:1063D000F1F71298812F8A95F1F71198812F8A95FC
:1063E000F1F7119A812F8A95F1F7129A812F8A95E8
:1063F000F1F71198812F8A95F1F7119A812F8A95DB
:10640000F1F71298812F8A95F1F71198812F8A95CB
:10641000F1F7119A812F8A95F1F7129811980A983D
:10642000802F8A95F1F780910A068D53823008F407
:10643000E9C080EE9EE20197F1F787ED9CE00E94B3
:1064400022190A9A119A129815E0812F8A95F1F76C
:106450001198812F8A95F1F7119A812F8A95F1F77A
:10646000129A812F8A95F1F71198812F8A95F1F769
:10647000119A812F8A95F1F71298812F8A95F1F759
:106480001198812F8A95F1F7119A812F8A95F1F74A
:106490001298812F8A95F1F71198812F8A95F1F73B
:1064A000119A812F8A95F1F71298812F8A95F1F729
:1064B0001198812F8A95F1F7119A812F8A95F1F71A
:1064C000129811980A9802E0802F8A95F1F78FEFC1
:1064D0009FE30E94811D0A9A119A129A812F8A9530
:1064E000F1F71198812F8A95F1F7119A812F8A95EA
:1064F000F1F7129A812F8A95F1F71198812F8A95D9
:10650000F1F7119A812F8A95F1F71298812F8A95C8
:10651000F1F71198812F8A95F1F7119A812F8A95B9
:10652000F1F7129A812F8A95F1F71198812F8A95A8
:10653000F1F7119A812F8A95F1F71298812F8A9598
:10654000F1F71198812F8A95F1F7119A812F8A9589
:10655000F1F7129811980A98802F8A95F1F7809197
:106560000A068D53823048F080EE9EE20197F1F7E3
:106570002F982A981F910F9108950A9A119A1298AC
:10658000812F8A95F1F71198812F8A95F1F7119A49
:10659000812F8A95F1F71298812F8A95F1F711983A
:1065A000812F8A95F1F7119A812F8A95F1F7129828
:1065B000812F8A95F1F71198812F8A95F1F7119A19
:1065C000812F8A95F1F7129A812F8A95F1F7119808
:1065D000812F8A95F1F7119A812F8A95F1F7129AF6
:1065E000812F8A95F1F71198812F8A95F1F7119AE9
:1065F000812F8A95F1F7129811980A98802F8A9521
:10660000F1F7B2CF0A9A119A1298812F8A95F1F771
:106610001198812F8A95F1F7119A812F8A95F1F7B8
:106620001298812F8A95F1F71198812F8A95F1F7A9
:10663000119A812F8A95F1F71298812F8A95F1F797
:106640001198812F8A95F1F7119A812F8A95F1F788
:10665000129A812F8A95F1F71198812F8A95F1F777
:10666000119A812F8A95F1F7129A812F8A95F1F765
:106670001198812F8A95F1F7119A812F8A95F1F758
:10668000129811980A98802F8A95F1F7D2CEEF923E
:10669000FF920F931F937B018C0120E030E040E0DC
:1066A0005FE40E94473688238CF0C801B70120E0E0
:1066B00030E040E05FE40E94BF340E9405379B0158
:1066C000AC01205030404040504806C0C801B701DE
:1066D0000E9405379B01AC01B901CA011F910F91BE
:1066E000FF90EF900895A0E0B0E0E9E7F3E30C94A9
:1066F0001E3CDC012B01FA019C91923008F439C157
:10670000EB018881823008F433C1943069F484301D
:1067100009F02FC111969C9111978981981709F45E
:1067200028C1A9E1B2E025C1843009F421C1823039
:10673000A9F4923009F01DC19A01AD0188E0EA0187
:106740000990AE01E90109929E018150C1F7E20171
:10675000898111969C918923818308C1923009F423
:1067600007C112962D903C901397EB018A819B8173
:106770001496AD90BD90CD90DC901797EC80FD8085
:106780000E811F819101281B390BB90137FF04C00D
:1067900066277727621B730B603271050CF061C0AE
:1067A000121613066CF537014801062E04C09694A4
:1067B0008794779467940A94D2F721E030E040E020
:1067C00050E004C0220F331F441F551F6A95D2F7B3
:1067D00021503040404050402E213F214023512342
:1067E000211531054105510521F021E030E040E05F
:1067F00050E079018A01E628F728082919293CC0C8
:10680000232BD1F1260E371E35014601062E04C07A
:1068100096948794779467940A94D2F721E030E0B5
:1068200040E050E004C0220F331F441F551F6A95FB
:10683000D2F721503040404050402A213B214C218A
:106840005D21211531054105510521F021E030E0A0
:1068500040E050E059016A01A628B728C828D92885
:106860000BC0821593052CF01C01AA24BB246501E2
:1068700003C0EE24FF24870111969C91D20111964A
:106880008C91981709F445C0992339F0A801970114
:106890002A193B094C095D0906C0A60195012E196C
:1068A0003F09400B510B57FD08C0118233822282F1
:1068B00024833583468357831DC081E081833382DF
:1068C000228288279927DC01821B930BA40BB50B2E
:1068D00084839583A683B7830DC0220F331F441F83
:1068E000551F248335834683578382819381019783
:1068F000938382832481358146815781DA01C901DE
:106900000197A109B1098F5F9F4FAF4FBF4328F394
:106910000BC0918333822282EA0CFB1C0C1D1D1DCF
:10692000E482F5820683178383E0808324813581A6
:106930004681578157FF1AC0C901AA2797FDA09524
:10694000BA2F81709070A070B070569547953795AA
:106950002795822B932BA42BB52B84839583A68319
:10696000B78382819381019693838283DF0101C083
:10697000D201CD01CDB7DEB7E2E10C943A3CA0E202
:10698000B0E0E5ECF4E30C942A3C69837A838B83D2
:106990009C832D833E834F835887E9E0EE2EF12CB4
:1069A000EC0EFD1ECE010196B7010E947D388E01CE
:1069B0000F5E1F4FCE010596B8010E947D388A896F
:1069C00091E089278A8BC701B801AE01475E5F4F0E
:1069D0000E9473330E94A837A096E6E00C94463CD0
:1069E000A0E2B0E0E6EFF4E30C942A3C69837A83FA
:1069F0008B839C832D833E834F835887F9E0EF2E52
:106A0000F12CEC0EFD1ECE010196B7010E947D38DF
:106A10008E010F5E1F4FCE010596B8010E947D3892
:106A2000C701B801AE01475E5F4F0E9473330E94F9
:106A3000A837A096E6E00C94463CA0E2B0E0E3E282
:106A4000F5E30C941E3C69837A838B839C832D83AE
:106A50003E834F835887CE010196BE01675F7F4F0B
:106A60000E947D38CE010596BE016F5E7F4F0E9469
:106A70007D389985923088F089898230C8F09430C9
:106A800019F4823051F404C0843029F4923081F436
:106A900089E192E0C6C0923049F420E09A858A8963
:106AA000981321E02A87CE010996BBC0823049F4B1
:106AB00020E09A858A89981321E02A8BCE0141969D
:106AC000B0C02D843E844F8458886D887E888F881E
:106AD000988CEE24FF248701AA24BB24650140E0A2
:106AE00050E060E070E0E0E0F0E0C10181709070A3
:106AF000892BE9F0E60CF71C081D191D9A01AB0162
:106B00002A0D3B1D4C1D5D1D80E090E0A0E0B0E033
:106B1000E614F7040805190520F481E090E0A0E0F0
:106B2000B0E0BA01A901480F591F6A1F7B1FAA0CC8
:106B3000BB1CCC1CDD1C97FE08C081E090E0A0E0EF
:106B4000B0E0A82AB92ACA2ADB2A3196E032F10538
:106B500049F0660C771C881C991C5694479437940E
:106B60002794C3CFFA85EA892B893C898B859C853C
:106B7000280F391F2E5F3F4F17C0CA0181709070D8
:106B8000892B61F016950795F794E79480E090E0E3
:106B9000A0E0B0E8E82AF92A0A2B1B2B7695679526
:106BA000579547952F5F3F4F77FDE7CF0CC0440FB8
:106BB000551F661F771F17FD4160EE0CFF1C001F5D
:106BC000111F21503040403090E0590790E0690794
:106BD00090E4790760F32B8F3C8FDB01CA018F773C
:106BE0009070A070B07080349105A105B10561F47A
:106BF00047FD0AC0E114F1040105110529F0405CCC
:106C00005F4F6F4F7F4F40781A8EFE1711F081E073
:106C10008A8F4D8F5E8F6F8F78A383E0898FCE012F
:106C200049960E94A837A096E2E10C943A3CA8E16C
:106C3000B0E0EDE1F6E30C942A3C69837A838B8320
:106C40009C832D833E834F83588789E0E82EF12C67
:106C5000EC0EFD1ECE010196B7010E947D388E011B
:106C60000F5E1F4FCE010596B8010E947D388985C1
:106C7000823040F08989823028F0C701B8010E9433
:106C8000F53801C08FEF6896E6E00C94463CA8E129
:106C9000B0E0EDE4F6E30C942A3C69837A838B83BD
:106CA0009C832D833E834F83588789E0E82EF12C07
:106CB000EC0EFD1ECE010196B7010E947D388E01BB
:106CC0000F5E1F4FCE010596B8010E947D38898561
:106CD000823040F08989823028F0C701B8010E94D3
:106CE000F53801C08FEF6896E6E00C94463CA8E1C9
:106CF000B0E0EDE7F6E30C942A3C69837A838B835A
:106D00009C832D833E834F83588789E0E82EF12CA6
:106D1000EC0EFD1ECE010196B7010E947D388E015A
:106D20000F5E1F4FCE010596B8010E947D38898500
:106D3000823040F08989823028F0C701B8010E9472
:106D4000F53801C081E06896E6E00C94463CA8E086
:106D5000B0E0EDEAF6E30C94273C9B01AC0183E044
:106D60008983DA01C9018827B7FD83959927AA2766
:106D7000BB27B82E211531054105510519F482E0D4
:106D800089833AC08823A9F0203080E0380780E06A
:106D9000480780E8580729F460E070E080E09FEC45
:106DA00030C0EE24FF248701E21AF30A040B150B0E
:106DB00002C079018A018EE1C82ED12CDC82CB82FF
:106DC000ED82FE820F831887C801B7010E945937F0
:106DD00001971816190684F4082E04C0EE0CFF1C47
:106DE000001F111F0A94D2F7ED82FE820F831887CD
:106DF000C81AD90ADC82CB82BA82CE0101960E94DF
:106E0000A8372896E9E00C94433CACE0B0E0EBE016
:106E1000F7E30C942E3C69837A838B839C83CE01A9
:106E20000196BE016B5F7F4F0E947D388D8182305D
:106E300061F1823050F1843021F48E81882351F148
:106E40002EC02F81388537FD20C06E812F3131054E
:106E50001CF06623F9F023C08EE190E0821B930BB7
:106E600029853A854B855C8504C0569547953795AD
:106E700027958A95D2F76623B1F0509540953095C5
:106E800021953F4F4F4F5F4F0EC020E030E040E074
:106E900050E009C02FEF3FEF4FEF5FE704C020E065
:106EA00030E040E050E8B901CA012C96E2E00C94D1
:106EB0004A3CEF92FF920F931F937B018C0180E07D
:106EC000E81680E0F80681E0080780E0180788F4FB
:106ED0008FEFE816F1040105110531F028F088E084
:106EE00090E0A0E0B0E017C080E090E0A0E0B0E06B
:106EF00012C080E0E81680E0F80680E0080781E034
:106F0000180728F088E190E0A0E0B0E004C080E13C
:106F100090E0A0E0B0E020E230E040E050E0281B4C
:106F2000390B4A0B5B0B04C016950795F794E79451
:106F30008A95D2F7F701EF5DFD4F8081281B31095B
:106F400041095109C9011F910F91FF90EF900895D8
:106F5000DF92EF92FF920F931F93FC01E480F58084
:106F600006811781D1808081823048F480E090E0F2
:106F7000A0E1B0E0E82AF92A0A2B1B2BA5C0843037
:106F800009F49FC0823021F4EE24FF24870105C05C
:106F9000E114F1040105110519F4E0E0F0E096C0F8
:106FA000628173819FEF623879070CF05BC022E841
:106FB0003FEF261B370B2A3131052CF020E030E063
:106FC00040E050E02AC0B801A701022E04C0769527
:106FD0006795579547950A94D2F781E090E0A0E035
:106FE000B0E004C0880F991FAA1FBB1F2A95D2F7D3
:106FF0000197A109B1098E219F21A023B1230097F8
:10700000A105B10521F081E090E0A0E0B0E09A0197
:10701000AB01282B392B4A2B5B2BDA01C9018F7767
:107020009070A070B07080349105A105B10539F45D
:1070300027FF09C0205C3F4F4F4F5F4F04C0215CCA
:107040003F4F4F4F5F4FE0E0F0E02030A0E03A07C5
:10705000A0E04A07A0E45A0710F0E1E0F0E079016F
:107060008A0127C06038710564F5FB01E158FF4FC4
:10707000D801C7018F779070A070B07080349105EF
:10708000A105B10539F4E7FE0DC080E490E0A0E071
:10709000B0E004C08FE390E0A0E0B0E0E80EF91E9D
:1070A0000A1F1B1F17FF05C016950795F794E79455
:1070B000319687E016950795F794E7948A95D1F76E
:1070C00005C0EE24FF248701EFEFF0E06E2F6795F7
:1070D00066276795902F9F77D794DD24D7948E2FBE
:1070E0008695492F462B582F5D29B701CA011F915C
:1070F0000F91FF90EF90DF900895FC01DB0140813C
:1071000051812281622F6F7770E0221F2227221F78
:107110009381892F880F822B282F30E0991F992780
:10712000991F11969C93119721153105A9F54115C9
:1071300051056105710511F482E037C082E89FEFC7
:1071400013969C938E9312979A01AB0167E0220FDE
:10715000331F441F551F6A95D1F783E08C930DC0F0
:10716000220F331F441F551F12968D919C91139728
:10717000019713969C938E931297203080E03807E6
:1071800080E0480780E4580758F314962D933D9308
:107190004D935C93179708952F3F310579F441156E
:1071A00051056105710519F484E08C93089564FF1D
:1071B00003C081E08C9312C01C9210C02F57304046
:1071C00013963C932E93129783E08C9387E0440FA1
:1071D000551F661F771F8A95D1F7706414964D93DB
:1071E0005D936D937C93179708951F93DC01FB01CA
:1071F0009C91923008F447C08081823008F443C0EB
:10720000943051F411961C91843099F58181682F46
:1072100070E0611B71093FC0843021F0923031F47D
:107220008230B9F18181882389F12DC011961C919A
:1072300011978230F1F081811817D9F412962D91AF
:107240003C911397828193818217930794F02817BA
:107250003907BCF014968D919D910D90BC91A02D95
:107260002481358146815781281739074A075B07F2
:1072700018F4112341F00AC082179307A407B50739
:1072800040F4112319F061E070E005C06FEF7FEF6B
:1072900002C060E070E0CB011F910895DC0101C0E5
:1072A0006D9341505040E0F70895AEE0B0E0EBE55B
:1072B000F9E30C942C3C0D891E8986E08C831A839B
:1072C00009838FEF9FE79E838D83CE014996AC01A2
:1072D0006F89788DCE0101960E9478392F8138858B
:1072E000020F131FF80110822E96E4E00C94483C24
:1072F000ABE0B0E0EEE7F9E30C941E3C3C012B015F
:107300005A01FC0117821682838181FD03C06FEF51
:107310007FEFC8C19AE0892E1E010894211C311C00
:10732000F3012381F20123FD859123FF81912F0138
:10733000882309F4B4C1853239F423FD859123FFF4
:1073400081912F01853229F4B30190E00E946D3BB9
:10735000E7CF982FDD24CC249924FFE1FD15D0F050
:107360009B3269F09C3228F4903259F0933291F4B8
:107370000EC09D3249F0903369F441E024C052E0E0
:10738000D52A84E0D82A28C098E0D92A25C0E0E18F
:10739000DE2A22C0D7FC29C0892F80538A3070F49E
:1073A000D6FE05C0989C902C1124980E15C0C89C40
:1073B000C02C1124C80EF0E2DF2A0EC09E3229F440
:1073C000D6FC6DC140E4D42A07C09C3619F450E8BD
:1073D000D52A02C0983649F4F20123FD959123FF86
:1073E00091912F01992309F0B8CF892F85548330CB
:1073F00018F08052833038F444E050E0A40EB51EFB
:107400005FE359830FC0933631F0933779F09335AA
:1074100009F056C020C0F5018081898342E050E028
:10742000A40EB51E710101E010E012C0F501E0806C
:10743000F180D6FC03C06FEF7FEF02C0692D70E0D2
:1074400042E050E0A40EB51EC7010E94623B8C01D1
:107450005FE7D52214C0F501E080F180D6FC03C0BF
:107460006FEF7FEF02C0692D70E042E050E0A40EA4
:10747000B51EC7010E94573B8C0150E8D52AD3FEA8
:1074800007C01AC0B30180E290E00E946D3BCA942D
:107490008C2D90E008171907A8F30EC0F701D7FC50
:1074A0008591D7FE81917F01B30190E00E946D3BF1
:1074B000C110CA94015010400115110579F7ECC0B4
:1074C000943611F0993671F5D7FE08C0F501E080C9
:1074D000F1800281138144E050E00AC0F50180810F
:1074E00091817C010027F7FC0095102F42E050E0CD
:1074F000A40EB51E5FE6D52217FF0AC010950095B1
:10750000F094E094E11CF11C011D111D80E8D82AC3
:107510002AE030E0A101C801B7010E94993BF82E92
:10752000F21840C0953729F41D2D1F7E2AE030E067
:107530001DC01D2D197F9F3661F0903720F49835BE
:1075400009F0ADC00FC0903739F0983709F0A7C0E7
:1075500004C028E030E00AC0106114FD146020E18E
:1075600030E004C014FD166020E132E017FF08C0CF
:10757000F501608171818281938144E050E008C00F
:10758000F50180819181BC0180E090E042E050E013
:10759000A40EB51EA1010E94993BF82EF2188FE7A8
:1075A000D82ED122D6FE0BC05EEFD522F91438F4C6
:1075B000D4FE07C0D2FC05C08FEED82202C01F2D1A
:1075C00001C0192DD4FE0DC0FE01EF0DF11D80810B
:1075D000803319F499EED92208C01F5FD2FE05C08E
:1075E00003C08D2D867809F01F5F0D2DD3FC14C0CC
:1075F000D0FE0FC01C1510F09F2C0BC09F2C9C0CB4
:10760000911A1C2D06C0B30180E290E00E946D3BF0
:107610001F5F1C15C0F304C01C1510F4C11A01C073
:10762000CC2404FF10C0B30180E390E00E946D3BC6
:1076300002FF1EC001FD03C088E790E002C088E59C
:1076400090E0B3010CC0802F867891F001FF02C05A
:107650008BE201C080E2D7FC8DE2B30190E00E9492
:107660006D3B06C0B30180E390E00E946D3B9A94AD
:10767000F914C0F3FA94F101EF0DF11DB30180810B
:1076800090E00E946D3BFF20A9F706C0B30180E2A5
:1076900090E00E946D3BCA94CC20C1F741CEF3012B
:1076A00066817781CB012B96E2E10C943A3CFC0198
:1076B0000590615070400110D8F7809590958E0F1D
:1076C0009F1F0895FC016150704001900110D8F790
:1076D000809590958E0F9F1F08950F931F93CF93C2
:1076E000DF938C01EB018B8181FF1BC082FF0DC0FA
:1076F0002E813F818C819D812817390764F4E881B0
:10770000F9810193F983E88306C0E885F985802F24
:107710000995892B31F48E819F8101969F838E83F9
:1077200002C00FEF1FEFC801DF91CF911F910F91A2
:107730000895FA01AA27283051F1203181F1E89407
:107740006F936E7F6E5F7F4F8F4F9F4FAF4FB1E054
:107750003ED0B4E03CD0670F781F891F9A1FA11D4F
:10776000680F791F8A1F911DA11D6A0F711D811D50
:10777000911DA11D20D009F468943F912AE0269F15
:1077800011243019305D3193DEF6CF010895462F74
:107790004770405D4193B3E00FD0C9F7F6CF462F55
:1077A0004F70405D4A3318F0495D31FD40524193BE
:1077B00002D0A9F7EACFB4E0A6959795879577957B
:1077C0006795BA95C9F700976105710508959B0102
:1077D000AC010A2E06945795479537952795BA958B
:1077E000C9F7620F731F841F951FA01D089597FB93
:1077F000092E07260AD077FD04D00CD006D0002031
:107800001AF4709561957F4F0895F6F790958195DC
:107810009F4F0895AA1BBB1B51E107C0AA1FBB1FA6
:10782000A617B70710F0A61BB70B881F991F5A950C
:10783000A9F780959095BC01CD0108952F923F92B4
:107840004F925F926F927F928F929F92AF92BF9270
:10785000CF92DF92EF92FF920F931F93CF93DF931C
:10786000CDB7DEB7CA1BDB0B0FB6F894DEBF0FBE79
:10787000CDBF09942A88398848885F846E847D84C6
:107880008C849B84AA84B984C884DF80EE80FD80C8
:107890000C811B81AA81B981CE0FD11D0FB6F8943E
:1078A000DEBF0FBECDBFED01089591110EC0803235
:1078B00019F089508550D0F7089591110895815697
:1078C0008A5108F480528558089599278827089589
:0478D000F894FFCF5A
:1078D4007479706520253032780A00255820000A12
:1078E400504553207361797320567070203D2025D4
:1078F400642E25642C50756C73652074696D652045
:107904003D202564206D73000A5045533A202564B8
:107914002C25642C25642C25642C25642C25642CAE
:1079240025642C25642C25642C25642C25642C25A5
:1079340064000A25686400756E6B6E6F776E00478D
:10794400414C323256313000000000006701000023
:107954000000000000000000000000000000000023
:1079640000000800000000000000010048496F0109
:10797400041718002C0084002C00C41608003D00D5
:107984003C003A000A001000DC011400010002006F
:1079940005000A0014001E00280032003C004600C6
:1079A40050005A006400C80000000000B116B01670
:1079B400B316B216B516B416B716B616B916B81667
:1079C400BB16BA16BD16BC16BF16BE16C116C01617
:1079D400C316C216253032580025303458203A09CF
:1079E4000025303458203A0900000000000000004F
:1079F4000000010202030303030404040404040456
:107A04000405050505050505050505050505050523
:107A14000506060606060606060606060606060603
:107A240006060606060606060606060606060606F2
:107A340006070707070707070707070707070707D3
:107A440007070707070707070707070707070707C2
:107A540007070707070707070707070707070707B2
:107A640007070707070707070707070707070707A2
:107A74000708080808080808080808080808080883
:107A84000808080808080808080808080808080872
:107A94000808080808080808080808080808080862
:107AA4000808080808080808080808080808080852
:107AB4000808080808080808080808080808080842
:107AC4000808080808080808080808080808080832
:107AD4000808080808080808080808080808080822
:107AE4000808080808080808080808080808080812
:027AF400080088
:00000001FF
